:020000040000FA
:100800000DEF15F058EF04F0E8CF60F0D8CF61F0AD
:10081000E0CF62F0EACF64F0E9CF63F0FACF65F0A1
:10082000FBCF66F0F8CF67F0F7CF68F0F6CF69F04E
:10083000F5CF6AF0F4CF6BF0F3CF6CF0010EE06E01
:10084000F2B410EF11F09DB09EA001D027EF12F08E
:10085000A0B2A1A201D03DEF12F0310E9D16020E02
:10086000A016320EA316010EB616000EB916000E13
:100870006016F296F298F096F0986BC0F4FF6CC098
:10088000F3FF67C0F8FF68C0F7FF69C0F6FF6AC0F2
:10089000F5FF64C0EAFF63C0E9FF65C0FAFF66C008
:1008A000FBFF62C0E0FF60C0E8FF61C0D8FF10003E
:1008B000010EE06EF8CF6DF0F7CF6EF0F6CF6FF06F
:1008C000F5CF70F0F4CF75F0F3CF76F0EACF72F099
:1008D000E9CF71F0E2CF74F0E1CF73F09DBA9EAA38
:1008E00001D0A4EF04F09DB89EA801D0E7EF04F07A
:1008F000A3B2A4A201D011EF05F0A3BAA4AA01D01B
:1009000052EF0CF0A3B8A4A801D09BEF0CF0B6B046
:10091000B7A001D0C5EF0CF0300E9F6E000EA26E96
:10092000320EA56E010EB86E000ED26E000EA96ECC
:10093000D08E800EF16EF06A9D6AA06AA36AB66AD4
:10094000B96A606AF26A1100CF6ACE6A050EBD6E9E
:100950009B0EBC6E076A9E90A49201920196019430
:10096000ABB0ABB40180ABB20180ABB2AB98AB889B
:10097000AE5001B011000DC1D9FFDF6E0D2BF86A2A
:10098000F76A0419D890E836F7361C0FF66ED8B01F
:10099000F72AAC0EF7260900F5500519046F090077
:1009A000F550056F6DC0F8FF6EC0F7FF6FC0F6FF22
:1009B00070C0F5FF75C0F4FF76C0F3FF72C0EAFFA8
:1009C00071C0E9FF74C0E2FF73C0E1FF1100CF6A9C
:1009D000CE6A030EBD6E840EBC6E9E90A4920192F0
:1009E000019601940D2B0F0E0D5D085DD8B408D053
:1009F000D8B00CD0FF0AD8B406D09D980188110059
:100A00000451AD6E11000551AD6E11000AC0D3F155
:100A10000DA0D38FD3C189FF0DC1D9FFDF50AD6EBB
:100A2000AED7CF6ACE6AA49201B673EF05F001B8D3
:100A300029D001A401B220D001B027D00551041162
:100A4000D8A423D0030E105DD8B437EF06F0100EF3
:100A5000105DD8B433EF06F0010E07D0020E05D0BA
:100A6000030E03D0040E01D0060E116F108F030E7B
:100A7000086F0F53D8B409D00186040EBD6E290E3D
:100A8000BC6E0BD0AE50AE5001980196610EBD6E9B
:100A9000610EBC6E01B4018200D0019001840F0E82
:100AA0000D6FABB2AB98AB88D36B0DA0D38FD3C116
:100AB00089FF9D8A9D98FF0E046F056F6DC0F8FF3A
:100AC0006EC0F7FF6FC0F6FF70C0F5FF75C0F4FF92
:100AD00076C0F3FF72C0EAFF71C0E9FF74C0E2FFA5
:100AE00073C0E1FF11000AB621B001D0AA850AB493
:100AF00021B201D0AA850AB221B401D0AA850AB0D8
:100B000021B601D0AA850ABA21B801D0AA850AB8AF
:100B100021BA01D0AA850ABC20B801D0AA850ABC96
:100B2000AA810AACAA89A8B342D0AAA180EF07F093
:100B3000AAA97DEF0BF0AAA50DEF08F0AA6B918C86
:100B4000918E0AA606D00A6A0A849198918A919C8D
:100B5000CAD70AA406D00A6A0A829188918A919C0F
:100B6000C2D70AA206D00A6A0A809198919A919EE9
:100B7000BAD70AA006D00A6A0A8A9188919A919EE9
:100B8000B2D70AAA06D00A6A0A889198918A919ED9
:100B9000AAD70AA806D00A6A0A8C9188918A919EDF
:100BA000A2D70A6A0A869188919A919C9CD721A023
:100BB000A99121A2A99321A4A99521A6A99721A829
:100BC000A99921AAA99B20A8A99D0AB6A9A101D0EB
:100BD0001ED00AB4A9A301D01AD00AB2A9A501D087
:100BE00016D00AB0A9A701D012D00ABAA9A901D07B
:100BF0000ED00AB8A9AB01D00AD00ABCA9AD01D069
:100C000006D0A951D8B4A8A701D0A86B8ED7A96BDC
:100C1000BA6BA86B0B0E0ABC7B0E0F6FA06F100E89
:100C2000106F500E116FF00E126FA26F000E136F47
:100C30000D0E146F1A0E156F010EE26E160EE16E98
:100C4000E00EE96E000EEA6E1A0EBB6FEE50E66E15
:100C5000BB2FFCD7210E086F9D9A9E9A9D889E9867
:100C6000A49206EF05F0960E066E3CEF05F0960E88
:100C7000066EA0510F5DD8A445EF05F0D890A135C0
:100C8000115DD8A445EF05F0100E0F5DD8B4B4D0B7
:100C90000B0E0F5DD8B405D17B0E0F5DD8B401D11A
:100CA000700E0F5DD8A43CEF05F0F66B20888E0E19
:100CB000A25DD8B41FD0B00EA25DD8B439D0BC0E9E
:100CC000A25DD8B467D0E60EA25DD8A43CEF05F0D3
:100CD00012C135F513C134F514C133F515C132F520
:100CE00016C1E8F417C1E7F418C16DF419C16CF42A
:100CF0003CEF05F013C16FF214C126F016C166F483
:100D000017C176F418C186F419C196F41AC1A6F475
:100D10001BC1B6F422C169F423C179F424C189F45A
:100D200025C199F426C1A9F427C1B9F43CEF05F017
:100D300012C16BF413C16AF414C165F415C164F4F3
:100D400016C163F417C162F418C161F419C160F4EB
:100D50001AC17BF41BC17AF41CC175F41DC174F473
:100D60001EC173F41FC172F420C171F421C170F46B
:100D700022C18BF423C18AF424C185F425C184F4F3
:100D800026C183F427C182F428C181F429C180F4EB
:100D90003CEF05F012C19BF413C19AF414C195F411
:100DA00015C194F416C193F417C192F418C191F4CB
:100DB00019C190F41AC1ABF41BC1AAF41CC1A5F46B
:100DC0001DC1A4F41EC1A3F41FC1A2F420C1A1F44B
:100DD00021C1A0F422C1BBF423C1BAF424C1B5F4EB
:100DE00025C1B4F426C1B3F427C1B2F428C1B1F4CB
:100DF00029C1B0F43CEF05F00AB6F06B0AB62180C9
:100E00000AB4F16B0AB421820AB2F26B0AB22184ED
:100E10000AB0F36B0AB021860ABAF46B0ABA2188C9
:100E20000AB8F56B0AB8218A2E0EA25DD8B41FD07D
:100E3000E90EA25DD8A43CEF05F0010EEA6E120E99
:100E4000E96E040EE26E0D0E0AB41D0E0AB22D0EEE
:100E50000AB03D0E0ABA4D0E0AB85D0EE16E0E0ED6
:100E6000D36FEE50E56ED32FFCD73CEF05F0010EAB
:100E7000EA6E120EE96E050EE26E050E0AB40D0E54
:100E80000AB2150E0AB01D0E0ABA250E0AB82D0EAA
:100E9000E16E060ED36FEE50E56ED32FFCD73CEF1C
:100EA00005F012C1A4F113C1A5F114C1A6F115C139
:100EB000A7F1A5ADA5BF01D03CEF05F0060EA5BD7D
:100EC000070EA86F010E0AB4020E0AB2040E0AB091
:100ED000080E0ABA100E0AB8200E0ABC400EBA6FED
:100EE000010EE26E120EE16E000EEA6EE00EE96E89
:100EF0001A0EBB6FE650EE6EBB2FFCD73CEF05F031
:100F0000100E0F6FA06FA351D8A40FD0030E106F57
:100F1000510E116FE90E126FA26F000E136F070EC4
:100F2000146FA16F060E09EF08F00AB621B001D0C8
:100F30006BD00AB421B201D067D00AB221B401D07B
:100F400063D00AB021B601D05FD00ABA21B801D06F
:100F50005BD00AB821BA01D057D0010EA35DD8A446
:100F60000FD0030E106F510E116F2E0E126FA26F65
:100F7000000E136F030E146FA16F060E09EF08F039
:100F8000020EA35DD8A441D0100E106F500E116F49
:100F9000180E126FA26F000E136F050E146F0A0E5B
:100FA000156F030EEA6E000E0AB4020E0AB2040EAA
:100FB0000AB0060E0ABA080E0AB80A0EE96EEECF9B
:100FC00016F1EECF17F1186B196B1A6B1C6B1D6BBA
:100FD00069C21EF1232C23C01EF122C01BF11F6B1E
:100FE000C80E1E5D010ED8B01F6FCA0E1E5DD8B4AC
:100FF0001F6B110E1E5D010ED8B41F6F1F511B1306
:101000001F6B110E09EF08F0AA85AA81A36B73EF7D
:1010100005F0086FA32B2CEF06F00B0E0ABC7B0E1D
:101020000F6FA06FA8A1A8B301D003D0A351D8B46B
:10103000A32BA351D8A40ED0030E106F510E116F25
:10104000F00E126FA26F000E136F0D0E146FA16FD2
:10105000060EDFD7010EA35DD8A4A1D0D76BD86B45
:10106000D96B96C0BBF1000EE26E970EE16E600E7A
:10107000E75CD8B4D7813F0EE75CD8B4D783300E95
:10108000E75CD8B4D785400EE75CD8B4D787500E5C
:10109000E75CD8B4D789200EE75CD8B4D78BB00E04
:1010A000E75CD8B4D881B10EE75CD8B4D883B20E6F
:1010B000E75CD8B4D885B30EE75CD8B4D887B40E53
:1010C000E75CD8B4D981B50EE75CD8B4D983B60E45
:1010D000E75CD8B4D985B70EE75CD8B4D987B80E29
:1010E000E75CD8B4D989B90EE75CD8B4D98BBA0E0D
:1010F000E75CD8B4D98DBB0EE75CD8B4D98FA00E0D
:10110000E75CD8B4D889A10EE65CD8B4D88BBB2FE5
:10111000AED7009CD7BB008C100E106F500E116F15
:10112000A00E126FA26F000E136F0D0E146F1A0E29
:10113000156F96C016F197C017F198C018F199C0B5
:1011400019F19AC01AF19BC01BF19CC01CF19DC003
:101150001DF19EC01EF19FC01FF1A0C020F1A1C0D3
:1011600021F1A2C022F1A3C023F1A4C024F1A5C0A3
:1011700025F1A6C026F1A7C027F1A8C028F1A9C073
:1011800029F1AAC02AF1ABC02BF1ACC02CF1ADC043
:101190002DF1AEC02EF1AFC02FF1210E3AD7050EC2
:1011A000A35DD8B0A6D2010EEA6EE26EAB0E0AB411
:1011B000AD0E0AB2AF0E0AB0B10E0ABAB30E0AB83B
:1011C000B50E0ABCB70EE96EE928E16ED00EEF5CF1
:1011D000D8B0EF6A160EEF5C470ED8B4D7B101D085
:1011E000EF6E240EEF5C470ED8B4E7B001D0EF6E7F
:1011F000470EEF5C850ED8B4D7B301D0EF6E530E17
:10120000EF5C660ED8B4E7B001D0EF6E660EEF5C0F
:10121000850ED7A5D7B701D0D8A401D0EF6E720E36
:10122000EF5C850ED8B4E7BC01D0EF6E850EEF5CA5
:101230008A0ED8B4D7B901D0EF6E8A0EEF5C930E48
:10124000D8B4D7BB01D0EF6E930EEF5C970ED8B435
:10125000D8B101D0EF6E970EEF5C9B0ED8B4D8B327
:1012600001D0EF6E9B0EEF5C9F0ED8B4D8B501D0C5
:10127000EF6E9F0EEF5CA30ED8B4D8B701D0EF6E1F
:10128000A30EEF5CA70ED8B4D9B101D0EF6EA70EB4
:10129000EF5CAB0ED8B4D9B301D0EF6EAB0EEF5C00
:1012A000AF0ED8B4D9B501D0EF6EAF0EEF5CB30E70
:1012B000D8B4D9B701D0EF6EB30EEF5CB70ED8B487
:1012C000D9B901D0EF6EB70EEF5CBB0ED8B4D9BB65
:1012D00001D0EF6EBB0EEF5CBF0ED8B4D9BD01D00C
:1012E000EF6EBF0EEF5CC30ED8B4D9BF01D0EF6E66
:1012F000C30EEF5CCD0ED8B4D8B901D0EF6ECD0ED1
:10130000EF5C000ED8B4D8B901D0EF6E460ED7B35B
:10131000650EEF5CD8B405D0840EEF5CD8B407D06E
:101320000CD0E7B2E790E782E7A0E79206D0E7BEED
:10133000E79CE78EE7ACE79E00D0EF50040D040E6B
:10134000F324F66ED8B0F42A770EF424F76EF86A18
:101350000900F5CFA4F10900F5CFA5F10900F5CFFB
:10136000A7F10900F5CFA6F1EFCFD6F1EF2A000ED5
:10137000E26E800EE16EA545BB6FA7C1D3F1A6C199
:10138000D4F1700EA45DD8B40FD1600EA45DD8B4B2
:1013900028D03F0EA45DD8B443D0300EA45DD8B49D
:1013A0005CD0500EA45DD8B478D0200EA45DD8B423
:1013B00092D0B00EA45DD8B49DD0B10EA45DD8B4C7
:1013C000A8D0B20EA45DD8B4B3D0B30EA45DD8B487
:1013D000BED0A00EA45DD8B4C9D0A10EA45DD8B46F
:1013E000D4D0D351040D000EF86EC40EF324F66E63
:1013F000D8B0F42A7A0EF424F76ED8B0F82A510E39
:10140000D45F000ED4B1040ED4B3060ED4B1D4A36D
:1014100001D0080ED4B50A0EF726D8B0F82AD2D0DB
:10142000D351040D000EF86E440EF324F66ED8B0BE
:10143000F42A880EF424F76ED8B0F82A560ED45F3A
:10144000D8A4C0D0800EF626D8B0F72AD8B0F82A93
:10145000020EF726D8B0F82AB5D0400ED7B7A46F41
:10146000D351040D000EF86E440EF324F66ED8B07E
:10147000F42A880EF424F76ED8B0F82A560ED45FFA
:10148000D8A4A0D0800EF626D8B0F72AD8B0F82A73
:10149000020EF726D8B0F82A95D0C80ED35D200EDC
:1014A000D8B0D35F500ED35D700ED8B0D35F300E7E
:1014B000D35D180ED8B0D35FD351040D000EF86E73
:1014C000440EF324F66ED8B0F42A940EF424F76E8A
:1014D000D8B0F82A77D0D351040D000EF86EA40EC0
:1014E000F324F66ED8B0F42A950EF424F76ED8B033
:1014F000F82A68D0D351040D000EF86E240EF324A0
:10150000F66ED8B0F42A970EF424F76ED8B0F82A05
:1015100059D0D351040D000EF86EA40EF324F66ECC
:10152000D8B0F42A970EF424F76ED8B0F82A4AD02F
:10153000D351040D000EF86E240EF324F66ED8B0CD
:10154000F42A980EF424F76ED8B0F82A3BD0D35181
:10155000040D000EF86EA40EF324F66ED8B0F42A33
:10156000980EF424F76ED8B0F82A2CD0D351040D7D
:10157000000EF86E240EF324F66ED8B0F42A9D0EF9
:10158000F424F76ED8B0F82A1DD0D351040D000E04
:10159000F86EA40EF324F66ED8B0F42A9D0EF4244F
:1015A000F76ED8B0F82A0ED0D351040D000EF86EA5
:1015B000040EF324F66ED8B0F42A6B0EF424F76E02
:1015C000D8B0F82A0900F5CFEAFF0900F5CFE9FF06
:1015D000EF50E66EBB2FF6D7160EBB6FA545BB5F6F
:1015E000D8B403D0E66ABB2FFDD7100E106F500E93
:1015F000116FF00E126FA26F000E136F0D0E146FAD
:101600001A0E156FA4C116F1A5C117F10F0E171709
:10161000A6C118F1A7C119F180C01AF181C01BF150
:1016200082C01CF183C01DF184C01EF185C01FF172
:1016300086C020F187C021F188C022F189C023F142
:101640008AC024F18BC025F18CC026F18DC027F112
:101650008EC028F18FC029F190C02AF191C02BF1E2
:1016600092C02CF193C02DF194C02EF195C02FF1B2
:10167000050ED65DD8A425D00AB60BC424F10AB64F
:101680000AC425F10AB41BC424F10AB41AC425F112
:101690000AB22BC424F10AB22AC425F10AB03BC411
:1016A00024F10AB03AC425F10ABA4BC424F10ABAAB
:1016B0004AC425F10AB85BC424F10AB85AC425F11A
:1016C00016D0060ED65DD8A412D0000E0AB627504A
:1016D0000AB428500AB229500AB02A500ABA2B502C
:1016E0000AB82C500A0DF4CF20F1F3CF21F1210ECE
:1016F00090D4AA85A36B73EF05F0700E0F6FA06FE7
:10170000A351D8A40FD0030E106F510E116F8E0E7F
:10171000126FA26F000E136F0B0E146FA16F060EE7
:1017200009EF08F020A8BAD0010EA35DD8A40FD00D
:10173000030E106F510E116FB00E126FA26F000EDC
:10174000136F0C0E146FA16F060E09EF08F0020E56
:10175000A35DD8A40FD0030E106F510E116FBC0EF5
:10176000126FA26F000E136F0C0E146FA16F060E96
:1017700009EF08F0030EA35DD8A40FD0030E106F7D
:10178000510E116FE60E126FA26F000E136F040E52
:10179000146FA16F060E09EF08F0040EA35DD8A424
:1017A00018D0100E106F500E116F050E126FA26F31
:1017B000000E136F020E146F040E156F0AC216F19D
:1017C00009C217F10CC218F10BC219F10B0E09EF87
:1017D00008F0050EA35DD8A441D0100E106F500E76
:1017E000116F1B0E126FA26F000E136F070E146F96
:1017F0000E0E156F52C016F142C217F169C218F1F0
:10180000232C23C018F122C019F11A6BC80E185DE1
:10181000010ED8B01A6FCA0E185DD8B41A6B110E2B
:10182000185D010ED8B41A6F1A511913800E0E10DC
:101830001A6F0FC01BF130C01CF133C01DF134C052
:101840001EF135C01FF132C020F131C021F138C086
:1018500022F139C023F1150E09EF08F0060EA35D41
:10186000D8A41CD0100E106F500E116F880E126F7E
:10187000A26F000E136F030E146F060E156FA6C233
:1018800016F1A7C217F1A8C218F1A9C219F1AAC28C
:101890001AF1ABC21BF10D0E09EF08F0AA89A36B78
:1018A00073EF05F00F0EE06EB36AB26A050E4B6F70
:1018B0009B0E4A6FA192B790096A02920296029417
:1018C00022B122B5028022B3028022B3229922895A
:1018D0001D5102B01100010EE06E1DCFE8FF0EC1D8
:1018E000D9FFDF6E0E2BF86AF76A0619D890E83632
:1018F000F7361C0FF66ED8B0F72AAC0EF7260900A3
:10190000F5500719066F0900F550076F6DC0F8FF15
:101910006EC0F7FF6FC0F6FF70C0F5FF75C0F4FF33
:1019200076C0F3FF72C0EAFF71C0E9FF74C0E2FF46
:1019300073C0E1FF11000F0EE06EB36AB26A030ECE
:101940004B6F840E4A6F010EE06EA192B790029227
:10195000029602940E2B570E0E5D095DD8B408D086
:10196000D8B00CD0FF0AD8B406D0A39802881100D2
:1019700006C11CFF110007C11CFF11008F800EC1A2
:10198000D9FFDFCF1CFFDF50AED7B36AB26AB79082
:1019900002B6B4D002B8A1D002A402B2A3D002B061
:1019A000A1D007510611D8A49DD0700E575DD8B4B0
:1019B00024EF0DF07B0E575DD8B443EF0EF0E70E29
:1019C000575DD8A472EF0DF0100E585DD8A472EFD9
:1019D0000DF0500E595DD8A472EF0DF0000E5A5D57
:1019E000D8A472EF0DF0A50E5E5DD8A472EF0DF0D5
:1019F0005A0E5F5DD8A472EF0DF0020EE06E036B1D
:101A0000FE0E626E030E636EFF0E616E7F9E7F9C04
:101A10007F84800EF16EF06A550E7E6EAA0E7E6E89
:101A20007F8204007FB2FDD7FF0E626E616E7F9EE3
:101A30007F9C7F84550E7E6EAA0E7E6E7F82040090
:101A40007FB2FDD715EF00F0030E585DD8B485EFD7
:101A50000DF0100E585DD8B4B9EF0DF0010E07D09F
:101A6000020E05D0030E03D0040E01D0060E596FEE
:101A7000588F030E096F5753D8B434D002860F0E17
:101A8000E06E040E4B6F290E4A6F010EE06E02905D
:101A90000284570E0E6F0F0EE06E22B32299228938
:101AA0008F90A38AA398010EE06EFF0E066F076F5A
:101AB0006DC0F8FF6EC0F7FF6FC0F6FF70C0F5FF96
:101AC00075C0F4FF76C0F3FF72C0EAFF71C0E9FF92
:101AD00074C0E2FF73C0E1FF11000F0EE06E1D51F4
:101AE0001D51029802960F0EE06E270E4B6F100EDE
:101AF0004A6F010EE06E02B40282C9D7A39AA49A7B
:101B0000A388A498B790BEEF0CF0570E0E5D08089E
:101B1000D8A472EF0DF0510E595DD8A472EF0DF0FC
:101B20005B53D8A430EF0DF05A055C25D8B030EFE8
:101B30000DF0960E086E5A0ED96E5C45D16F596F36
:101B4000030F096F5A51040D040EF324F66ED8B03A
:101B5000F42A6B0EF424F76EF86A0900F5CFEAFF59
:101B60000900F5CFE9FFEF50DE6ED12FF6D73EEF3B
:101B70000DF0570E0E5D096F090E095DD8A072EFCA
:101B80000DF05D5DD8A472EF0DF0900E595DD8B4E4
:101B900038D0500E595DD8A472EF0DF05D415A2532
:101BA000D8B030EF0DF05B53D8A432EF0DF05C45A8
:101BB0005D5DD8A432EF0DF0960E086E5A51080DF7
:101BC000040EF324F66ED8B0F42A6F0EF424F76EE8
:101BD000F86A5E0ED96E0900F5CFEAFF0900F5CF6D
:101BE000E9FFDE50EF6E0900F5CFEAFF0900F5CFFF
:101BF000E9FF010EEF6E5D2FEED7060E096F3EEF87
:101C00000DF0090E5A5DD8A472EF0DF05B53D8A405
:101C100032EF0DF05C455D5DD8A432EF0DF0010EA2
:101C20005C5DD8A472EF0DF05A0E5E5DD8A472EF21
:101C30000DF0A50E5F5DD8A472EF0DF00F0EE06EF3
:101C4000AC6A216BAB6A226BF26AF16AF06A030E2E
:101C5000636EF00E626EC30E616E7F9E7F9C7F840A
:101C6000550E7E6EAA0E7E6E7F8204007FB2FDD777
:101C7000F10E626E3C0E616E550E7E6EAA0E7E6E89
:101C80007F8200EF00F0030E585DD8B4C4EF10F06F
:101C9000100E585DD8A42EEF0DF0570E0E5D096F93
:101CA000090E095DD8A072EF0DF05D5DD8A472EF4A
:101CB0000DF0500E595DD8A472EF0DF05D415A251C
:101CC000D8B030EF0DF05B53D8A432EF0DF05C4587
:101CD0005D5DD8A432EF0DF0960E086E5A51080DD6
:101CE000040EF324F66ED8B0F42A6F0EF424F76EC7
:101CF000F86A5E0ED96E0900F5CFEAFF0900F5CF4C
:101D0000E9FFDE50EF6E0900F5CFEAFF0900F5CFDD
:101D1000E9FF010EEF6E5D2FEED7060E096FF00E94
:101D20005A5DD8A43EEF0DF0030EE26E800EE16E18
:101D3000A8A7A8A530D0E0C0D3F1D351C65DD8A4E0
:101D40002AD0E3C0D3F1D351C95DD8A424D0C6C1F1
:101D5000E0F0C7C1E1F0C8C1E2F0C9C1E3F0000E94
:101D6000EA6EE40EE96E1A0ED16FE650EE6ED12FD8
:101D7000FCD7A887A895BAB1A981BAB3A983BAB587
:101D8000A985BAB7A987BAB9A989BABBA98BBABDBF
:101D9000A98D3EEF0DF0C745D16FC9C1D3F1C8C1C0
:101DA000D4F1700EC65DD8B43EEF0DF03F0EC65DA7
:101DB000D8B476D0300EC65DD8B498D0400EC65D8B
:101DC000D8B494D0200EC65DD8B4B6D0B00EC65DDF
:101DD000D8B4C1D0B10EC65DD8B4CCD0B20EC65DF9
:101DE000D8B4D7D0B30EC65DD8B4E2D0B40EC65DB9
:101DF000D8B4EDD0B50EC65DD8B4F8D0B60EC65D79
:101E0000D8B403D1B70EC65DD8B40ED1B80EC65D36
:101E1000D8B419D1B90EC65DD8B424D1BA0EC65DF6
:101E2000D8B42FD1BB0EC65DD8B43AD1A00EC65DD2
:101E3000D8B445D1A10EC65DD8B450D1500EC65D00
:101E4000D8B45BD1D351040D000EF86EC40EF32448
:101E5000F66ED8B0F42A7A0EF424F76ED8B0F82AC9
:101E6000510ED45F000ED4B1040ED4B3060ED4B11B
:101E7000D4A301D0080ED4B50A0EF726D8B0F82A9C
:101E8000D4A558D1AD0ED35DD8A454D1AC81AE81C8
:101E9000B081B281B481B681B881FC6BFD6B4AD14F
:101EA000D351040D000EF86E440EF324F66ED8B034
:101EB000F42A880EF424F76ED8B0F82A560ED45FB0
:101EC000D8A438D1800EF626D8B0F72AD8B0F82A90
:101ED000020EF726D8B0F82AAC81AE81B081B2816B
:101EE000B481B681B881FC6BFD6B24D1D351040D54
:101EF000000EF86E440EF324F66ED8B0F42A8E0E5F
:101F0000F424F76ED8B0F82A560ED45FD8A412D1B4
:101F1000800EF626D8B0F72AD8B0F82A020EF72697
:101F2000D8B0F82AAC8DAE8DB08DB28DB48DB68D93
:101F3000B88DFC6BFD6BFED0D351040D000EF86E16
:101F4000A40EF324F66ED8B0F42A950EF424F76E9E
:101F5000D8B0F82AEFD0D351040D000EF86E240E3D
:101F6000F324F66ED8B0F42A970EF424F76ED8B0A6
:101F7000F82AE0D0D351040D000EF86EA40EF3241D
:101F8000F66ED8B0F42A970EF424F76ED8B0F82A7B
:101F9000D1D0D351040D000EF86E240EF324F66E4A
:101FA000D8B0F42A980EF424F76ED8B0F82AC2D02C
:101FB000D351040D000EF86EA40EF324F66ED8B0C3
:101FC000F42A980EF424F76ED8B0F82AB3D0D3517F
:101FD000040D000EF86E240EF324F66ED8B0F42A29
:101FE000990EF424F76ED8B0F82AA4D0D351040D7A
:101FF000000EF86EA40EF324F66ED8B0F42A990EF3
:10200000F424F76ED8B0F82A95D0D351040D000E01
:10201000F86E240EF324F66ED8B0F42A9A0EF42447
:10202000F76ED8B0F82A86D0D351040D000EF86EA2
:10203000A40EF324F66ED8B0F42A9A0EF424F76EA8
:10204000D8B0F82A77D0D351040D000EF86E240EC4
:10205000F324F66ED8B0F42A9B0EF424F76ED8B0B1
:10206000F82A68D0D351040D000EF86EA40EF324A4
:10207000F66ED8B0F42A9B0EF424F76ED8B0F82A86
:1020800059D0D351040D000EF86E240EF324F66ED1
:10209000D8B0F42A9C0EF424F76ED8B0F82A4AD0AF
:1020A000D351040D000EF86EA40EF324F66ED8B0D2
:1020B000F42A9C0EF424F76ED8B0F82A3BD0D35102
:1020C000040D000EF86E240EF324F66ED8B0F42A38
:1020D0009D0EF424F76ED8B0F82A2CD0D351040DFD
:1020E000000EF86EA40EF324F66ED8B0F42A9D0EFE
:1020F000F424F76ED8B0F82A1DD0C80ED35D200E98
:10210000D8B0D35F500ED35D700ED8B0D35F300E11
:10211000D35D180ED8B0D35FD351040D000EF86E06
:10212000440EF324F66ED8B0F42A940EF424F76E1D
:10213000D8B0F82A0900F5CFEAFF0900F5CFE9FF8A
:10214000E650EF6ED12FF6D73EEF0DF0D351080DCC
:10215000000EF86E040EF324F66ED8B0F42A6F0E5B
:10216000F424F76ED8B0F82A5E0ED96E0900F5CFC8
:10217000EAFF0900F5CFE9FFE650EF6E090009001C
:10218000D12FF4D73EEF0DF0570E0E5D0808D8A4FE
:1021900072EF0DF0510E595DD8A472EF0DF05B5344
:1021A000D8A430EF0DF05A055C25D8B030EF0DF013
:1021B000960E086E5A0ED96EF00E5A5DD8A412D043
:1021C000A8A510D0000EEA6EE00EE96E5C45D16F56
:1021D000596F030F096FEE50DE6ED12FFCD7A89117
:1021E0003EEF0DF05A0ED96E5C45D16F596F030F5B
:1021F000096F5A51040D040EF324F66ED8B0F42A78
:102200006B0EF424F76EF86A0900F5CFEAFF0900B7
:10221000F5CFE9FFEF50DE6ED12FF6D73EEF0DF090
:10222000F294E093E0B1E083E09181B0E081070EA9
:10223000E117FB6A220EFA6EE145420FD8B0FA2A86
:10224000F96ECCD0D5D0D9D0DAD0DED0DFD0EAD07C
:10225000FCD0E09FE24BE207640EE261E08F052ACA
:10226000560E055CD8A03DEF04F0056AE8B1EAA17E
:1022700001D00DD0E8A1EAB101D009D0E9A102D086
:10228000E99109D0E8A1EA91E8B1EA8104D0E7A197
:10229000E991E7B1E981E8B3EAA301D00DD0E8A361
:1022A000EAB301D009D0E9A302D0E99309D0E8A3A9
:1022B000EA93E8B3EA8304D0E7A3E993E7B3E983B9
:1022C000E8B5EAA501D00DD0E8A5EAB501D009D05E
:1022D000E9A502D0E99509D0E8A5EA95E8B5EA852F
:1022E00004D0E7A5E995E7B5E985E8B7EAA701D005
:1022F0000DD0E8A7EAB701D009D0E9A702D0E99745
:1023000009D0E8A7EA97E8B7EA8704D0E7A7E997F2
:10231000E7B7E987E8B9EAA901D00DD0E8A9EAB999
:1023200001D009D0E9A902D0E99909D0E8A9EA9930
:10233000E8B9EA8904D0E7A9E999E7B9E989E8BBEE
:10234000EAAB01D00DD0E8ABEABB01D009D0E9ABD4
:1023500002D0E99B09D0E8ABEA9BE8BBEA8B04D04A
:10236000E7ABE99BE7BBE98BE9A19092E9B19082E9
:10237000E9A38D94E9B38D84E9A58D98E9B58D889D
:10238000E9A78D9CE9B78D8CE9A99190E9B9918075
:10239000E9AB9194E9BB9184EAA19090EAB1908075
:1023A000EAA38D96EAB38D86EAA58D9AEAB58D8A61
:1023B000EAA78D9EEAB78D8EEAA99192EAB9918239
:1023C000EAAB9196EABB9186E7AD8A94E7BD8A8431
:1023D000E7AF8A96E7BF8A863DEF04F0E0B1E0A35D
:1023E00038D7E12BE095130EE261E085E26B31D73F
:1023F000E12BE46B81B2E4892CD7E12B2AD7E0A151
:10240000E0B327D7E12B25D7E12B23D7E12BE34BF3
:10241000E307060EE0B5050EE35DD8A01AD7E36B1F
:10242000008017D7E12B81B2E48984A0E48184A2E3
:10243000E48387A6E48587A4E48786A6E48BE45139
:10244000E55FD8B4E66FE56F04D7E16B02D79E90E5
:10245000270EBD6E100EBC6E019601900184FF0E1A
:10246000046F056F0F0E0D6FEB6B0DA0EB8FEBC1C3
:1024700089FF9D8A9D983DEF04F0A1920F0EE06EBA
:10248000270E4B6F100E4A6F010EE06E02960290FF
:102490000284FF0E066F076F570E0E6F8F90A38A90
:1024A000A3983DEF04F00900F550E06F0900F550E6
:1024B000636E0900F550626E0900F550E26F090085
:1024C000F550E16F0900F550E46F0900F550E36F36
:1024D0000900F550E66F0900F550E56F0900F55069
:1024E000E76F0900F550E86F0900F550E96F090042
:1024F000F550EA6F0900F550EB6F0900F550EC6FED
:102500001200616E7F9E7F9C7F84F29E550E7E6ED0
:10251000AA0E7E6E7F82F28E1200EDC2F8F202D019
:10252000EFC2F8F2FA6BE951F85DD8A0FA81F851E0
:10253000EB5DD8A0FA811200EDC2F8F2EEC2F9F21A
:1025400004D0EFC2F8F2F0C2F9F2FA6BEA51F95D89
:10255000D8A005D0D8A404D0E951F85DD8A0FA815C
:10256000F951EC5DD8A005D0D8A404D0F851EB5DAA
:10257000D8A0FA811200E96E040EEA6E0B0EE26E2C
:10258000000EE16E0C0E186EEE50E66E182EFCD7A3
:102590000D6B0F6B0E6B106B146B156B010E0BBF7D
:1025A0000A6F0BBF0B6B06A306B701D006B901D0AB
:1025B00089D01E0E0427D8B0052B0B51055DD8A07D
:1025C00081D0D8A404D00A51045DD8A07BD00A5190
:1025D000045FD8A005070B51055F04510553D8A42B
:1025E000FF0E0F6F040E0F5DD8A01295070E0F5D42
:1025F000D8B01285090E0F5DD8A012930C0E0F5D96
:10260000D8B012830E0E0F5DD8A01291110E0F5D7F
:10261000D8B01281140E0F5FD8A00F6B0F51D8B431
:102620001197040E0F5DD8B01187030E0F5DD8A06F
:102630001195060E0F5DD8B01185050E0F5DD8A05F
:102640001193080E0F5DD8B01183090E0F5DD8A04D
:102650003FD00D6F0A0E0F5DD8B0D8B43CD01181B9
:102660001851D890D8B4D88018350D03F3501927D5
:10267000D8B01A2BF4501A2718B316D018A129D0A5
:10268000D89033303324020F0D5D129DD8B0128DD7
:10269000030E3302D890F332D890F330020F0D5D61
:1026A000129FD8B0128F17D0020E33240D5D129DE9
:1026B000D8B0128DD8903330020F0D5D129FD8B074
:1026C000128F09D0129512931291119711951193AF
:1026D0001191129D129F06A506B700B864D01E0E78
:1026E000025FD8A0030703510B5DD8A05CD0D8A42B
:1026F00004D002510A5DD8A056D002510A5FD8A07A
:102700000B0703510B5F0A510B53D8A4FF0E106F38
:10271000040E105DD8A0129B070E105DD8B0128B6E
:10272000090E105DD8A012990C0E105DD8B0128958
:102730000E0E105DD8A01297110E105DD8B0128742
:10274000140E105FD8A0106B1051D8B4119F040E56
:10275000105DD8B0118F030E105DD8A0119D060E2C
:10276000105DD8B0118D050E105DD8A0119B080E1C
:10277000105DD8B0118B090E105DD8A01AD00E6F65
:102780000A0E105DD8B0D8B415D011891851D89060
:10279000D8B4D88018350E03F3501B27D8B01C2BA3
:1027A000F4501C2707D0129B12991297119F119D6C
:1027B000119B119911BF129511BF129311BF129164
:1027C00011B7129B11B7129911B712970151095DF8
:1027D000280F06AD320E156F290E155DD8B0139F68
:1027E000270E155DD8A0138F0051095D3C0F06AF71
:1027F000320E146F0D0EE96E0B0EEA6E0C51E16E87
:10280000090E186EEE50E66E182EFCD712000C5111
:10281000E96E0B0EEA6E090E186EEE6A182EFDD7E1
:102820001200020DF3CF18F0090DF350300FE96ECE
:102830000B0EEA6EEE5017B9EE50196E18500D0FD0
:10284000E96E020EEA6EEE501A6EEE501902F3CFE8
:102850005CF0F4CF5DF01A501902F3CF5BF0F45046
:102860005C26D8B05D2A4BC25EF04CC25FF0C1EC72
:1028700014F05B502227D8B0232B5C502327120082
:10288000020DF3CF18F0090DF350320FE96E0B0E65
:10289000EA6EEE5017B9EE50D0D7186A1A6A1B6A62
:1028A00027512A11D8B46CD027A107D09D511B26DF
:1028B0009C511A26D8B01B2A182A27A307D09F514B
:1028C0001B269E511A26D8B01B2A182A27A507D0E6
:1028D000A1511B26A0511A26D8B01B2A182A27A7B7
:1028E00007D0A3511B26A2511A26D8B01B2A182A9A
:1028F00027A907D0A5511B26A4511A26D8B01B2AF8
:10290000182A27AB07D0A7511B26A6511A26D8B0E4
:102910001B2A182A2AA107D0A9511B26A8511A261A
:10292000D8B01B2A182A2AA307D0AB511B26AA51BC
:102930001A26D8B01B2A182A2AA507D0AD511B2663
:10294000AC511A26D8B01B2A182A2AA707D0AF5193
:102950001B26AE511A26D8B01B2A182A2AA907D03E
:10296000B1511B26B0511A26D8B01B2A182A2AABFF
:1029700007D0B3511B26B2511A26D8B01B2A182AE9
:102980001200180E586E596A5A6AD8905B365C3637
:102990005D3659365A365F505A5CD8A00DD0D8A44F
:1029A00004D05E50595CD8A007D05B805E50595E61
:1029B000D8A05A065F505A5E582EE7D7D8905F329B
:1029C0005E325F505A5CD8A01200D8A404D05E508A
:1029D000595CD8A012005B2AD8B05C2A1200180EED
:1029E000586E596A5A6AD8905B365C365D365936ED
:1029F0005A365F505A5CD8A00DD0D8A404D05E508F
:102A0000595CD8A007D05B805E50595ED8A05A06AA
:102A10005F505A5E582EE7D71200E06AFE6B000E38
:102A2000FC6FC80EFB6F700EFD6F010EE06E700E36
:102A3000006F020EE06E006B016BFE0E626E030E05
:102A4000636E7F9E7F9C7F80C30E615CD8B44ED046
:102A5000FF0E626E030E636E7F9E7F9C7F80C30EAF
:102A6000615CD8B443D06C0EF66E9E0EF76E000E0D
:102A7000F86E53EC12F004007FB2FDD7E75181EC01
:102A800012F0E0A319D004007FB2FDD7624A632A96
:102A9000E75181EC12F004007FB2FDD7624A632A4D
:102AA000E85181EC12F004007FB2FDD7624A632A3C
:102AB000E85181EC12F00AD0E0A108D004007FB206
:102AC000FDD7624A632AE75181EC12F004007FB21D
:102AD000FDD70900004B012B000E015DD8A0C9D71E
:102AE000D8A404D0DB0E005DD8A0C3D704007FB209
:102AF000FDD7006B016B6C0EF66E9E0EF76E000E2E
:102B0000F86E7F9E7F9C53EC12F009007F8061502D
:102B1000ED6F624A632AE0A351D07F806150EF6F6E
:102B2000624A632A7F806150EE6F624A632A7F8027
:102B30006150F06F624A632AED51EF5DD8A404D072
:102B4000EE51F05DD8B417D0E5C2E9FFE6C2EAFF66
:102B5000010EEE6EEF6E9CEC12F0FAA10CD0EFC2FB
:102B6000EDF2F0C2EEF29CEC12F0FAA104D0E7C252
:102B7000EDF2E8C2EEF200510111D8A40ED0ED51F1
:102B8000EE19D8B40AD0EDC2EEF2EF51F019D8A484
:102B900004D0EFC2EDF2F0C2EEF2E1C2E9FFE2C210
:102BA000EAFFED51EE6EEE51EF6EE3C2E9FFE4C2D3
:102BB000EAFFED51EE6EEE51EF6E28D0E0A11BD092
:102BC0007F806150EF6F624A632AED51EF5DD8B4A8
:102BD00012D0E5C2E9FFE6C2EAFF010EEF6E8DEC0E
:102BE00012F0FAA108D0EFC2EDF28DEC12F0FAA1CA
:102BF00002D0E7C2EDF2E1C2E9FFE2C2EAFFED5125
:102C0000EF6EE3C2E9FFE4C2EAFFEF6E004B012B77
:102C1000000E015DD8A077D7D8A404D0DB0E005DEC
:102C2000D8A071D7006B016B960E086E000E996FDD
:102C3000640E986F070E9B6FD00E9A6F960E6A6F98
:102C4000000E55B0800E0E6E9D6AA06AA36AB66A29
:102C5000B96A606AF26A800EF16EF06ACF6ACE6A73
:102C6000270EBD6E100EBC6E010EDA6E010EE06E08
:102C70000F0E0D6F570E0E6FC66AC56A676A666AD9
:102C8000610EAC6ED10EAB6E080E656E670EAF6E48
:102C9000000ED46E9D8A0F0EE06E610E216FD10E74
:102CA000226F080E206F670E1E6F000E1F6FA38A23
:102CB000300E9F6E000EA26E320EA56E010EB86E23
:102CC000000ED26E000EA96ED08EC00EF26E010EF6
:102CD000D16E0400FC6A109010920F0EE06E000E90
:102CE000926EC30E936EC30E9416000E956E030E75
:102CF000966E600E976E2E0E986E0C0E996E000EEC
:102D00009A6E010EC212000EC16EBA0EC06E000E97
:102D1000256F0C0E246F000E236FC30ED56E310E7F
:102D2000CD6E310EB16E0A0EBB120A0EBB16000E2E
:102D30004E13000E4E170A0E49130A0E4917776AF2
:102D4000746A716A6E6A466B436B406B400E2D6FFE
:102D5000C66AC56A676A666A310E9D16210E9D12A3
:102D6000020EA016020EA012320EA316220EA312FD
:102D7000010EB66E010EB612000EB916000EB91293
:102D8000000E6016000E6012300E9F6E000EA26ED6
:102D9000320EA56E010EB86E000ED26E000EA96E38
:102DA000F06A800EF16EE00EF212E70EF216670E78
:102DB000AF62AF6E000ED462D46EACB4AC94ACAA69
:102DC000AC8AACB8AC98ACACAC8CACA0AC80D10E3E
:102DD000AB12AB96670E1E631E6F000E1F631F6F54
:102DE00021B5219521AB218B21B9219921AD218DCF
:102DF00021A12181D10E22132297E06AFE6B010EE0
:102E0000FA6F000EFC6FC80EFB6F700EFD6F010EA7
:102E1000E06E700E006FE0AF10D0F26AF16AF06AF7
:102E2000896A8A6A8B6A8C6A8D6A8E6A8F6A906AEE
:102E3000916A0400030000EF00F0170EFD5DD8A0BA
:102E40000ED0700ED8B4FC5DD8A009D0AC81AE8194
:102E5000B081B281B481B681B881FC6BFD6B020E8A
:102E6000E06EE6C103F00BC0E7F10CC0E8F10F0E15
:102E70000314046F0850D8A41DD0640E276E286E6A
:102E8000296E2A6E2B6E2C6EA06FA16FA26FA36F9E
:102E9000A46FA56F416B41C242F2316A326A306A57
:102EA000346A356A386A396A576A010E236E226AB3
:102EB000800E0E16320EFC5DD8B00DD0050EFC5DF6
:102EC000D8A009D003BA07D00EBE05D000B202D0F8
:102ED000008201D0009203AAFC6B0EBEFC6B320E86
:102EE000FC5DD8B0048003AA0891640EFC5DD8B0E4
:102EF00008B108D00881800E701B711BFAC020F346
:102F0000FAC021F3DFC418F009BD0AAD18AE06D02F
:102F1000708D718DFAC020F3FAC021F309AD0ABD9E
:102F200018BE06D0709D719DFAC020F3FAC021F33F
:102F3000FE0E09170A17E951D8B404D055B0FAC0EB
:102F40008DF555900EBE55B003D05580FAC08DF565
:102F500063C7B8F200BC5BCDB8F20EA4ADC7B8F23F
:102F600062C7B9F200BC5ACDB9F20EA4ACC7B9F22F
:102F70006BC7BAF200BC63CDBAF20EA4B1C7BAF205
:102F80006AC7BBF200BC62CDBBF20EA4B0C7BBF2F5
:102F90006FC7BCF200BC67CDBCF20EA4B1C7BCF2D7
:102FA0006EC7BDF200BC66CDBDF20EA4B0C7BDF2C7
:102FB000090EBD5DD8A009D0D8A405D0C40EBC5D53
:102FC000D8A4D8A002D0BC6BBD6B090EBB5DD8A045
:102FD00009D0D8A405D0C40EBA5DD8A4D8A002D018
:102FE000BA6BBB6B090EB95DD8A009D0D8A405D0C7
:102FF000C40EB85DD8A4D8A002D0B86BB96BBCC25F
:10300000BEF2BDC2BFF2BF51BB5DD8A00AD0D8A4EA
:1030100004D0BE51BA5DD8A004D0BAC2BEF2BBC2C1
:10302000BFF2BF51B95DD8A00AD0D8A404D0BE5118
:10303000B85DD8A004D0B8C2BEF2B9C2BFF2BE51CA
:10304000BF11D8B49AC2BEF2D8B49BC2BFF261C756
:10305000B0F200BC59CDB0F20EA4ABC7B0F260C75D
:10306000B1F200BC58CDB1F20EA4AAC7B1F269C743
:10307000B2F200BC61CDB2F20EA4AFC7B2F268C723
:10308000B3F200BC60CDB3F20EA4AEC7B3F26DC70D
:10309000B4F200BC65CDB4F20EA4AFC7B4F26CC7F5
:1030A000B5F200BC64CDB5F20EA4AEC7B5F2090E00
:1030B000B55DD8A009D0D8A405D0C40EB45DD8A4FD
:1030C000D8A002D0B46BB56B090EB35DD8A009D0FF
:1030D000D8A405D0C40EB25DD8A4D8A002D0B26BDB
:1030E000B36B090EB15DD8A009D0D8A405D0C40E29
:1030F000B05DD8A4D8A002D0B06BB16BB4C2B6F2A8
:10310000B5C2B7F2B751B35DD8A006D0D8A408D0E5
:10311000B651B25DD8B004D0B2C2B6F2B3C2B7F203
:10312000B751B15DD8A006D0D8A408D0B651B05DD3
:10313000D8B004D0B0C2B6F2B1C2B7F25D6AB7C2BD
:103140005CF0B6C25BF05F6A320E5E6EEFEC14F0BC
:103150005950D8A45B2A5B50190DF3CFB6F2F4CFC7
:10316000B7F2B751D8A405D0640EB65D640ED8A0EE
:10317000B66F9B51B75DD8A00BD0D8A405D09A519B
:10318000B65DD8B0D8B404D09AC2B6F29BC2B7F23A
:10319000B6C298F2B7C299F299510E5DD8A011D07B
:1031A000D8A404D098510D5DD8A00BD09B510E5DD2
:1031B000D8A00FD0D8A405D09A510D5DD8B0D8B4FE
:1031C00008D099C275F298C274F2FAC024F3FAC01A
:1031D00025F39951105DD8A011D0D8A404D09851EE
:1031E0000F5DD8A00BD09B51105DD8A00FD0D8A4F4
:1031F00005D09A510F5DD8B0D8B408D099C277F2F3
:1032000098C276F2FAC026F3FAC027F39951125DFC
:10321000D8A011D0D8A404D09851115DD8A00BD05B
:103220009B51125DD8A00FD0D8A405D09A51115D42
:10323000D8B0D8B408D099C279F298C278F2FAC05E
:1032400028F3FAC029F39951145DD8A011D0D8A45D
:1032500004D09851135DD8A00BD09B51145DD8A019
:103260000FD0D8A405D09A51135DD8B0D8B408D0E7
:1032700099C27BF298C27AF2FAC02AF3FAC02BF311
:103280009951165DD8A011D0D8A404D09851155DDD
:10329000D8A00BD09B51165DD8A00FD0D8A405D0D4
:1032A0009A51155DD8B0D8B408D099C27DF298C2B1
:1032B0007CF2FAC02CF3FAC02DF39951185DD8A016
:1032C00011D0D8A404D09851175DD8A00BD09B5131
:1032D000185DD8A00FD0D8A405D09A51175DD8B0EA
:1032E000D8B408D099C27FF298C27EF2FAC02EF309
:1032F000FAC02FF399511A5DD8A011D0D8A404D0E8
:103300009851195DD8A00BD09B511A5DD8A00FD051
:10331000D8A405D09A51195DD8B0D8B408D099C2B4
:1033200081F298C280F2FAC030F3FAC031F39951B9
:103330001C5DD8A011D0D8A404D098511B5DD8A092
:103340000BD09B511C5DD8A00FD0D8A405D09A51AA
:103350001B5DD8B0D8B408D099C283F298C282F26B
:10336000FAC032F3FAC033F399511E5DD8A011D0E0
:10337000D8A404D098511D5DD8A00BD09B511E5DE0
:10338000D8A00FD0D8A405D09A511D5DD8B0D8B41C
:1033900008D099C285F298C284F2FAC034F3FAC018
:1033A00035F39951205DD8A011D0D8A404D09851FC
:1033B0001F5DD8A00BD09B51205DD8A00FD0D8A402
:1033C00005D09A511F5DD8B0D8B408D099C287F201
:1033D00098C286F2FAC036F3FAC037F39951225DEB
:1033E000D8A011D0D8A404D09851215DD8A00BD07A
:1033F0009B51225DD8A00FD0D8A405D09A51215D51
:10340000D8B0D8B408D099C289F298C288F2FAC06C
:1034100038F3FAC039F39951245DD8A011D0D8A45B
:1034200004D09851235DD8A00BD09B51245DD8A027
:103430000FD0D8A405D09A51235DD8B0D8B408D005
:1034400099C28BF298C28AF2FAC03AF3FAC03BF3FF
:103450000C0E425DD8B002D042C241F20C0E415D6A
:10346000D8B0416B41C242F2008A0EA0009A30509F
:10347000D8A434BC01D0009A650EA05DD8B004D0A9
:103480000EAE00BAA0C227F0650E275C640ED8B05D
:10349000276E27C0A0F2650EA15DD8B004D00EAE95
:1034A00000BAA1C228F0650E285C640ED8B0286E60
:1034B00028C0A1F2650EA25DD8B004D00EAE00BA4D
:1034C000A2C229F0650E295C640ED8B0296E29C00D
:1034D000A2F2650EA35DD8B004D00EAE00BAA3C2AE
:1034E0002AF0650E2A5C640ED8B02A6E2AC0A3F2B8
:1034F000650EA45DD8B004D00EAE00BAA4C22BF005
:10350000650E2B5C640ED8B02B6E2BC0A4F2650E3A
:10351000A55DD8B004D00EAE00BAA5C22CF0650EE1
:103520002C5C640ED8B02C6E2CC0A5F2650EA65D86
:10353000D8B003D000BAA6C23AF0650E3A5C640E69
:10354000D8B03A6E3AC0A6F2650EA75DD8B003D0E7
:1035500000BAA7C23BF0650E3B5C640ED8B03B6E70
:103560003BC0A7F2650EA85DD8B003D000BAA8C2D0
:103570003CF0650E3C5C640ED8B03C6E3CC0A8F2DA
:10358000650EA95DD8B003D000BAA9C23DF0650EA2
:103590003D5C640ED8B03D6E3DC0A9F2650EAA5DDB
:1035A000D8B003D000BAAAC23EF0650E3E5C640EED
:1035B000D8B03E6E3EC0AAF2650EAB5DD8B003D067
:1035C00000BAABC23FF0650E3F5C640ED8B03F6EF0
:1035D0003FC0ABF2960E03B86A6F00966A51D8B43A
:1035E0000086010EE06E5A0EF05DD8B021905A0EA2
:1035F000F15DD8B021925A0EF25DD8B021945A0EE6
:10360000F35DD8B021965A0EF45DD8B021985A0EC9
:10361000F55DD8B0219A21C025F0960EF65DD8B0A0
:10362000209820A8266A20A8FEC0E8F420A8FEC0A2
:103630006DF420A8FEC06CF40850D8A414D0010E7C
:10364000186E18C096F0700E196E19C097F0000E23
:10365000EA6E980EE96EAF0EE95CD8A4D8A001D04E
:1036600002D0EE6AF8D7020EE06E00A0E1D0009022
:103670000650D8A406060850D8A408066A51D8A453
:103680006A07514B5107524B5207534B53074F4B4D
:103690004F07FC4BFC0754515511D8A4010E545F41
:1036A000D8A0555F56515711D8A4010E565FD8A027
:1036B000575F58515911D8A4010E585FD8A0595FCF
:1036C0005A515B11D8A4010E5A5FD8A05B5F5C51C0
:1036D0005D11D8A4010E5C5FD8A05D5F5E515F11E3
:1036E000D8A4010E5E5FD8A05F5F010EE06EEC4BC8
:1036F000EC07090EEC650DD0EC6BF04BF007F14BCD
:10370000F107F24BF207F34BF307F44BF407F54BD9
:10371000F507F64BF607FC4BFD2BD8B4FD07040E5E
:10372000E06EC04BC007C14BC107C24BC207C34BC1
:10373000C307C44BC407C54BC507C64BC607C74B19
:10374000C707C84BC807C94BC907CA4BCA07CB4BE9
:10375000CB07D04BD007D14BD107D24BD207D34B9D
:10376000D307D44BD407D54BD507D64BD607D74B69
:10377000D707D84BD807D94BD907DA4BDA07DB4B39
:10378000DB07E22BD8B4E32BD8B4E307E42BD8B49F
:10379000E52BD8B4E507E64BE607EA2BD8B4EB2BCC
:1037A000D8B4EB07EE2BD8B4EF2BD8B4EF07F02B3F
:1037B000D8B4F12BD8B4F107F22BD8B4F32BD8B48A
:1037C000F307F42BD8B4F52BD8B4F507F62BD8B4FF
:1037D000F72BD8B4F707F82BD8B4F92BD8B4F907DE
:1037E0000B0EE06E1E511F11D8A4010E1E5FD8A053
:1037F0001F5F20512111D8A4010E205FD8A0215FA6
:10380000C04BC007C14BC107C24BC207C34BC30764
:10381000C44BC407C54BC507C64BC607C74BC70734
:10382000C84BC807C94BC907CA4BCA07CB4BCB0704
:10383000020EE06E7FB283D1056B066B6C0EF66EE6
:103840009E0EF76E000EF86E53EC12F0E5C2E9FF23
:10385000E6C2EAFFEF50D8A40ED00900054B062BB4
:10386000000E065DD8A0F0D7D8A467D0DB0E055DAA
:10387000D8A0EAD762D0E0B321D0EF6AE3C2E9FF73
:10388000E4C2EAFFE1C2E1FFE2C2E2FFEF50ED6F06
:103890008DEC12F0FAA103D0E750EF6E4ED0EF504E
:1038A000E76E81EC12F0E0A14AD104007FB2FDD7AF
:1038B000624A632AEF5081EC12F041D1EE6AEF6A5E
:1038C000E3C2E9FFE4C2EAFFE1C2E1FFE2C2E2FFD4
:1038D000F29EEE50ED6FEF50EE6FF28E9CEC12F018
:1038E000FAA105D0E650EE6EE750EF6E26D00051FB
:1038F0000111D8A404D0ED51EE19D8A4F3D7ED519D
:10390000E66E81EC12F004007FB2FDD7624A632AB2
:10391000ED5181EC12F004007FB2FDD7624A632AB8
:10392000EE51E76E81EC12F004007FB2FDD7624ADF
:10393000632AEE5181EC12F002D1000EF86E0051B4
:10394000100D6C0EF324F66ED8B0F42A9E0EF424FB
:10395000F76ED8B0F82A0151100DF350F726D8B001
:10396000F82AF450F82653EC12F07F806150ED6F86
:10397000624A632AE0B358D0E0A143D07F8061500F
:10398000EF6F8DEC12F0FAB10CD0ED51EF5DD8B4C1
:1039900038D0E1C2E9FFE2C2EAFFEF50ED5DD8B4F2
:1039A00029D090EC12F0FAB10BD0E1C2E9FFE2C2EB
:1039B000EAFFEF50EF5DD8A403D0EFC2EDF21AD0CA
:1039C0008DEC12F0FAA116D090EC12F0FAB103D0FF
:1039D000EFC2EDF20FD0E1C2E9FFE2C2EAFFEF5021
:1039E000F86F92EC12F0FAB103D0F8C2EDF202D007
:1039F000E7C2EDF2E5C2E9FFE6C2EAFF010EEF6EB3
:103A000007D0E5C2E9FFE6C2EAFFEF50D8A489D0AB
:103A1000E1C2E9FFE2C2EAFFED51EF6EE3C2E9FF66
:103A2000E4C2EAFFEF6E7DD07F806150EF6F624AA3
:103A3000632A7F806150EE6F624A632A7F80615003
:103A4000F06F624A632A9CEC12F0FAB116D0ED5185
:103A5000EF5DD8A404D0EE51F05DD8B44AD0E1C2F5
:103A6000E9FFE2C2EAFFEE50F86FEF50EE5DD8A436
:103A700004D0F851ED5DD8B434D0A1EC12F0FAB115
:103A80000ED0E1C2E9FFE2C2EAFFEE50F86FEF505C
:103A9000F05DD8A404D0F851EF5DD8B422D09CECEE
:103AA00012F0FAA11ED0A1EC12F0FAB105D0EFC2CB
:103AB000EDF2F0C2EEF215D0E1C2E9FFE2C2EAFF98
:103AC000EE50F86FEF50F96FA5EC12F0FAB105D097
:103AD000F8C2EDF2F9C2EDF204D0E7C2EDF2E8C2AD
:103AE000EEF2E5C2E9FFE6C2EAFF010EEE6EEF6E0E
:103AF0000AD0E5C2E9FFE6C2EAFFEE50D8A411D031
:103B0000EF50D8A40ED0E1C2E9FFE2C2EAFFE3C25F
:103B1000E1FFE4C2E2FFED51EE6EE66EEE51EF6EB4
:103B2000E76E004B012B000E015DD8A008D0D8A491
:103B300004D0DB0E005DD8A002D0006B016B040E38
:103B4000E06E00940098009E22BE008E010E186E5A
:103B50000EBE3DD20B510A11D8A425A00BD00BBF2D
:103B600005D0060E0B5DD8B005D006D0FE0E0B5D5D
:103B7000D8B002D0C06B2D90960EC05DD8B02D800D
:103B80001B511A11D8A425A20BD01BBF05D0060EBD
:103B90001B5DD8B005D006D0FE0E1B5DD8B002D09C
:103BA000C16B2D92960EC15DD8B02D822B512A117A
:103BB000D8A425A40BD02BBF05D0060E2B5DD8B002
:103BC00005D006D0FE0E2B5DD8B002D0C26B2D946E
:103BD000960EC25DD8B02D843B513A11D8A425A6CB
:103BE0000BD03BBF05D0060E3B5DD8B005D006D04C
:103BF000FE0E3B5DD8B002D0C36B2D96960EC35D12
:103C0000D8B02D864B514A11D8A425A80BD04BBF54
:103C100005D0060E4B5DD8B005D006D0FE0E4B5D2C
:103C2000D8B002D0C46B2D98960EC45DD8B02D8844
:103C30005B515A11D8A425AA0BD05BBF05D0060E44
:103C40005B5DD8B005D006D0FE0E5B5DD8B002D06B
:103C5000C56B2D9A960EC55DD8B02D8A6B516A1131
:103C6000D8A426A00BD06BBF05D0060E6B5DD8B0D4
:103C700005D006D0FE0E6B5DD8B002D0C66B2E907C
:103C8000960EC65DD8B02E807B517A11D8A426A29C
:103C90000BD07BBF05D0060E7B5DD8B005D006D01B
:103CA000FE0E7B5DD8B002D0C76B2E92960EC75D1C
:103CB000D8B02E828B518A11D8A426A40BD08BBFEA
:103CC00005D0060E8B5DD8B005D006D0FE0E8B5DFC
:103CD000D8B002D0C86B2E94960EC85DD8B02E8492
:103CE0009B519A11D8A426A60BD09BBF05D0060ED7
:103CF0009B5DD8B005D006D0FE0E9B5DD8B002D03B
:103D0000C96B2E96960EC95DD8B02E86AB51AA11FE
:103D1000D8A426A80BD0ABBF05D0060EAB5DD8B09B
:103D200005D006D0FE0EAB5DD8B002D0CA6B2E987F
:103D3000960ECA5DD8B02E88BB51BA11D8A426AA57
:103D40000BD0BBBF05D0060EBB5DD8B005D006D0EA
:103D5000FE0EBB5DD8B002D0CB6B2E9A960ECB5D1B
:103D6000D8B02E8A0951D8B404D0650E095DD8A008
:103D700002D0D06BDC91960ED05DD8B0DC811951A9
:103D8000D8B404D0650E195DD8A002D0D16BDC93F5
:103D9000960ED15DD8B0DC832951D8B404D0650E1D
:103DA000295DD8A002D0D26BDC95960ED25DD8B03A
:103DB000DC853951D8B404D0650E395DD8A002D065
:103DC000D36BDC97960ED35DD8B0DC874951D8B45D
:103DD00004D0650E495DD8A002D0D46BDC99960E54
:103DE000D45DD8B0DC895951D8B404D0650E595D82
:103DF000D8A002D0D56BDC9B960ED55DD8B0DC8BFD
:103E00006951D8B404D0650E695DD8A002D0D66BD4
:103E1000DD91960ED65DD8B0DD817951D8B404D04D
:103E2000650E795DD8A002D0D76BDD93960ED75D75
:103E3000D8B0DD838951D8B404D0650E895DD8A08F
:103E400002D0D86BDD95960ED85DD8B0DD8599513E
:103E5000D8B404D0650E995DD8A002D0D96BDD9797
:103E6000960ED95DD8B0DD87A951D8B404D0650EBF
:103E7000A95DD8A002D0DA6BDD99960EDA5DD8B0D4
:103E8000DD89B951D8B404D0650EB95DD8A002D08F
:103E9000DB6BDD9B960EDB5DD8B0DD8BDEB1DCB17C
:103EA00001D02FD0DEB3DCB301D02BD0DEB5DCB532
:103EB00001D027D0DEB7DCB701D023D0DEB9DCB922
:103EC00001D01FD0DEBBDCBB01D01BD0E0B1DDB127
:103ED00001D017D0E0B3DDB301D013D0E0B5DDB52C
:103EE00001D00FD0E0B7DDB701D00BD0E0B9DDB91C
:103EF00001D007D0E0BBDDBB01D003D0E46BE56BA4
:103F00000F9C0651161126113611461156116611D5
:103F1000761186119611A611B611C00BD8B4E46FB4
:103F2000D8B4E56F04A0E46B04A0E56B070EE55D73
:103F3000D8A009D0080ED8B4E45DD8A004D0120EE1
:103F4000186E00840F8CDEB12DB001D02FD0DEB3FF
:103F50002DB201D02BD0DEB52DB401D027D0DEB7E5
:103F60002DB601D023D0DEB92DB801D01FD0DEBBD5
:103F70002DBA01D01BD0E0B12EB001D017D0E0B3E4
:103F80002EB201D013D0E0B52EB401D00FD0E0B7DF
:103F90002EB601D00BD0E0B92EB801D007D0E0BBCF
:103FA0002EBA01D003D0E26BE36B0F9A04A0E26B50
:103FB00004A0E36B070EE35DD8A009D0080ED8B4C7
:103FC000E25DD8A004D0110E186E0F8A008E25A0D5
:103FD00053900DBF1BD00D510C11D8B40BD0EE6B0C
:103FE000EF6B060E0D5DD8A025A001D05380D8B090
:103FF000539016D00B0EEF5DD8A012D0D8A404D0E9
:10400000B80EEE5DD8A00CD053900AD0EE6BEF6BDB
:10401000FE0E0D5DD8A05390D8B025A001D05380DE
:1040200025A253921DBF1BD01D511C11D8B40BD01B
:10403000F06BF16B060E1D5DD8A025A201D0538256
:10404000D8B0539216D00B0EF15DD8A012D0D8A4E0
:1040500004D0B80EF05DD8A00CD053920AD0F06B0B
:10406000F16BFE0E1D5DD8A05392D8B025A201D0F1
:10407000538225A453942DBF1BD02D512C11D8B49D
:104080000BD0F26BF36B060E2D5DD8A025A401D0EA
:104090005384D8B0539416D00B0EF35DD8A012D031
:1040A000D8A404D0B80EF25DD8A00CD053940AD096
:1040B000F26BF36BFE0E2D5DD8A05394D8B025A4FF
:1040C00001D0538425A653963DBF1BD03D513C11D2
:1040D000D8B40BD0F46BF56B060E3D5DD8A025A6C9
:1040E00001D05386D8B0539616D00B0EF55DD8A0EC
:1040F00012D0D8A404D0B80EF45DD8A00CD053963A
:104100000AD0F46BF56BFE0E3D5DD8A05396D8B087
:1041100025A601D0538625A853984DBF1BD04D51DD
:104120004C11D8B40BD0F66BF76B060E4D5DD8A0D2
:1041300025A801D05388D8B0539816D00B0EF75D40
:10414000D8A012D0D8A404D0B80EF65DD8A00CD058
:1041500053980AD0F66BF76BFE0E4D5DD8A05398BE
:10416000D8B025A801D0538825AA539A5DBF1BD08B
:104170005D515C11D8B40BD0F86BF96B060E5D5D28
:10418000D8A025AA01D0538AD8B0539A16D00B0EC6
:10419000F95DD8A012D0D8A404D0B80EF85DD8A08C
:1041A0000CD0539A0AD0F86BF96BFE0E5D5DD8A067
:1041B000539AD8B025AA01D0538A040EE06E04B0F9
:1041C000048E04B018D0040EEB5DD8A014D0D8A48F
:1041D000048ED8A404D0B00EEA5DD8B0048E050ECB
:1041E000EB5DD8A008D0D8A40480D8A404D0DC0EFD
:1041F000EA5DD8B004800EBE0F940EBE0F9E0EBEB8
:104200000F9A0EBE67D0196A21B0198021B21982A7
:1042100021B4198421B6198621B8198821BA198ABE
:1042200020B8198E19C0DEF426C0E0F4DE51DF1983
:10423000DE15D8B404D0DE51DF13FAC04AF3E051E2
:10424000E119E015D8B404D0E051E113FAC04BF302
:10425000E951D8B409D0DEC4DFF4E0C4E1F4FAC017
:104260004AF3FAC04BF3E96BDE51DF193F0BD8A4D8
:1042700004D0E051E119D8B407D004A005D0CA0E8B
:10428000186E0F84008E01D00F94DEAFDFAF07D021
:1042900004A005D0CB0E186E0F86008E01D00F96AD
:1042A00000A60F9000B60F80E8B10F82E8A10F9230
:1042B00004A00F9004A00F92DFAF0FA001D00F82D7
:1042C0000FA00FB2008E0F9E25502610D8B404A068
:1042D00001D00F8E0850D8A4E66B960EE65DD8B0DC
:1042E00004A00AD0CC0E0EBECB0E186E0EAE0F88F8
:1042F0000EBE0F86008E03D00F980EBE0F96C80E0E
:104300000FA00FB2186ECD0E0EBE20A801D0186EF1
:10431000E7C41AF0CD0E1A5CCD0ED8B4186E18C0D2
:1043200069F257500EBE0F12186A0FB00FA201D0DB
:104330000EBE01D0182A0EBE00A601D0182A18C041
:1043400068F2010E0FBC070E0FBA060E0FB4030E73
:104350000FB6040E0FB8050E0FA00FB2020E186EA6
:1043600018C0F7F23050D8A40EA001D034BC01D050
:10437000008E0EBEBAEF30F006511611261136111E
:10438000461156116611761186119611A611B611B5
:10439000100BD8A400883050D8A434BC35AA01D062
:1043A00022A001D000880B0EE06E2B6B2C6B1E0E32
:1043B000B417D8A42B81B517D8A42B83B617D8A4CB
:1043C0002B85B717D8A42B87B817D8A42B89B91772
:1043D000D8A42B8BBA17D8A42C81BB17D8A42C83B4
:1043E000BC17D8A42C85BD17D8A42C87BE17D8A479
:1043F0002C89BF17D8A42C8B06C4B4FB16C4B5FBFC
:1044000026C4B6FB36C4B7FB46C4B8FB56C4B9FBDA
:1044100066C4BAFB76C4BBFB86C4BCFB96C4BDFBBA
:10442000A6C4BEFBB6C4BFFB22A02D911E0EB415C0
:10443000D8B42BA101D02D811E0EB515D8B42BA355
:1044400001D02D811E0EB615D8B42BA501D02D811B
:104450001E0EB715D8B42BA701D02D811E0EB8158E
:10446000D8B42BA901D02D811E0EB915D8B42BAB11
:1044700001D02D811E0EBA15D8B42CA101D02D81EA
:104480001E0EBB15D8B42CA301D02D811E0EBC1559
:10449000D8B42CA501D02D811E0EBD15D8B42CA7E3
:1044A00001D02D811E0EBE15D8B42CA901D02D81AE
:1044B0001E0EBF15D8B42CAB01D02D810AC218F046
:1044C00018AE00BE30EF2FF0196B1A6B1B6B1C6B14
:1044D00025A0C06B300E0C6FC80EC05DD8B02DA0EB
:1044E0000CD025C218FB34CB11FB35CB12FB36CBDD
:1044F00013FB000EBBEC12F002D007EC14F025A267
:10450000C16B390E0C6FC80EC15DD8B02DA20CD096
:1045100026C218FB3DCB11FB3ECB12FB3FCB13FB5E
:10452000100EBBEC12F002D007EC14F025A4C26B05
:10453000420E0C6FC80EC25DD8B02DA40CD027C29D
:1045400018FB46CB11FB47CB12FB48CB13FB200ECD
:10455000BBEC12F002D007EC14F025A6C36B4B0E97
:104560000C6FC80EC35DD8B02DA60CD028C218FBA6
:104570004FCB11FB50CB12FB51CB13FB300EBBECDE
:1045800012F002D007EC14F025A8C46B540E0C6F87
:10459000C80EC45DD8B02DA80CD029C218FB58CBCA
:1045A00011FB59CB12FB5ACB13FB400EBBEC12F0A4
:1045B00002D007EC14F025AAC56B5D0E0C6FC80E77
:1045C000C55DD8B02DAA0CD02AC218FB61CB11FB57
:1045D00062CB12FB63CB13FB500EBBEC12F002D08C
:1045E00007EC14F026A0C66B660E0C6FC80EC65DF5
:1045F000D8B02EA00CD02BC218FB6ACB11FB6BCB12
:1046000012FB6CCB13FB600EBBEC12F002D007EC7C
:1046100014F026A2C76B6F0E0C6FC80EC75DD8B022
:104620002EA20CD02CC218FB73CB11FB74CB12FB47
:1046300075CB13FB700EBBEC12F002D007EC14F03C
:1046400026A4C86B780E0C6FC80EC85DD8B02EA417
:104650000CD02DC218FB7CCB11FB7DCB12FB7ECB8B
:1046600013FB800EBBEC12F002D007EC14F026A670
:10467000C96B810E0C6FC80EC95DD8B02EA60CD0C8
:104680002EC218FB85CB11FB86CB12FB87CB13FB0D
:10469000900EBBEC12F002D007EC14F026A8CA6B07
:1046A0008A0E0C6FC80ECA5DD8B02EA80CD02FC2CF
:1046B00018FB8ECB11FB8FCB12FB90CB13FBA00E04
:1046C000BBEC12F002D007EC14F026AACB6B930ED1
:1046D0000C6FC80ECB5DD8B02EAA0CD030C218FB20
:1046E00097CB11FB98CB12FB99CB13FBB00EBBEC15
:1046F00012F002D007EC14F0000E25B0341125B2F0
:104700003D1125B4461125B64F1125B8581125BACB
:10471000611126B06A1126B2731126B47C1126B637
:10472000851126B88E1126BA9711166F000E25B086
:10473000351125B23E1125B4471125B6501125B8C3
:10474000591125BA621126B06B1126B2741126B424
:104750007D1126B6861126B88F1126BA9811C00B86
:104760002EB1010947B83F0B2E6F04A0166B04A0B1
:104770002E6B34501D5DD8B404D0B80E1E6F0B0ED6
:104780001F6F34C01DFB04A01E6B04A01F6B04A090
:10479000206B04A0216B04A038D03050D8B404D0D2
:1047A0001E511F11D8A431D01A511C5DD8A017D0AA
:1047B000D8A406D019511B5DD8A011D0D8B425D0EB
:1047C00017B923D020512111D8A416A101D01DD092
:1047D000100E176F280E206F230E216F16D017B101
:1047E00014D020512111D8A416A901D00ED02EBD6D
:1047F00006D00EB217A901D016A901D006D0010E1D
:10480000176F280E206F230E216FBC0E496E020E0B
:10481000486EDA0E4B6E020E4A6E020EE06E4B6B65
:104820004C6B25A006D00D514B27D8B04C2B0E5108
:104830004C2725A206D00F514B27D8B04C2B105136
:104840004C2725A406D011514B27D8B04C2B125120
:104850004C2725A606D013514B27D8B04C2B14510A
:104860004C2725A806D015514B27D8B04C2B1651F4
:104870004C2725AA06D017514B27D8B04C2B1851DE
:104880004C2726A006D019514B27D8B04C2B1A51D3
:104890004C2726A206D01B514B27D8B04C2B1C51BD
:1048A0004C2726A406D01D514B27D8B04C2B1E51A7
:1048B0004C2726A606D01F514B27D8B04C2B205191
:1048C0004C2726A806D021514B27D8B04C2B22517B
:1048D0004C2726AA06D023514B27D8B04C2B245165
:1048E0004C270B0EE06E226B236B256B286B175148
:1048F0001615D8B49ED017513415D8B404D0000E74
:1049000011EC14F0258117513D15D8B404D0010ED7
:1049100011EC14F0258317514615D8B404D0020EBB
:1049200011EC14F0258517514F15D8B404D0030E9F
:1049300011EC14F0258717515815D8B404D0040E83
:1049400011EC14F0258917516115D8B404D0050E67
:1049500011EC14F0258B17516A15D8B404D0060E4B
:1049600011EC14F0288117517315D8B404D0070E38
:1049700011EC14F0288317517C15D8B404D0080E1C
:1049800011EC14F0288517518515D8B404D0090E00
:1049900011EC14F0288717518E15D8B404D00A0EE4
:1049A00011EC14F0288917519715D8B404D00B0EC8
:1049B00011EC14F0288B42C218F017B91ED03050F9
:1049C000D8A434BC01D034BE01D009D02351D8A41E
:1049D00006D0020E225DD8B002D0020E226F48C06F
:1049E00042F02251495C436ED8A042062351425CFA
:1049F000010E4326D8B0422AB1D13050D8A434AEEB
:104A000001D009D02351D8A406D0020E225DD8B01F
:104A100002D0020E226F4AC042F022514B24436E54
:104A2000D8B0422A23514224010E435ED8A0420648
:104A300095D100B8179117B9C9D016A316B501D0F2
:104A4000179117A1AFEF2DF016A360D034B32581D5
:104A500034A703D0000E40EC14F03DB325833DA7EE
:104A600003D0010E40EC14F046B3258546A703D0D1
:104A7000020E40EC14F04FB325874FA703D0030E6E
:104A800040EC14F058B3258958A703D0040E40EC2D
:104A900014F061B3258B61A703D0050E40EC14F030
:104AA0006AB328816AA703D0060E40EC14F073B3F2
:104AB000288373A703D0070E40EC14F07CB328853D
:104AC0007CA703D0080E40EC14F085B3288785A797
:104AD00003D0090E40EC14F08EB328898EA703D0C2
:104AE0000A0E40EC14F097B3288B97A703D00B0E57
:104AF00040EC14F048C042F02251495C436ED8A00B
:104B000042060A0E4326D8B0422A28D134B5258160
:104B100034A703D0000E40EC14F03DB525833DA72B
:104B200003D0010E40EC14F046B5258546A703D00E
:104B3000020E40EC14F04FB525874FA703D0030EAB
:104B400040EC14F058B5258958A703D0040E40EC6A
:104B500014F061B5258B61A703D0050E40EC14F06D
:104B60006AB528816AA703D0060E40EC14F073B52D
:104B7000288373A703D0070E40EC14F07CB528857A
:104B80007CA703D0080E40EC14F085B5288785A7D4
:104B900003D0090E40EC14F08EB528898EA703D0FF
:104BA0000A0E40EC14F097B5288B97A703D00B0E94
:104BB00040EC14F048C042F02251495C436ED8A04A
:104BC00042060A0E4326D8B0422AC8D016AB16BDFC
:104BD00001D0179917A9AFEF2DF016AB60D034BBF9
:104BE000258134AF03D0000E40EC14F03DBB25838B
:104BF0003DAF03D0010E40EC14F046BB258546AF17
:104C000003D0020E40EC14F04FBB25874FAF03D00A
:104C1000030E40EC14F058BB258958AF03D0040EA6
:104C200040EC14F061BB258B61AF03D0050E40EC66
:104C300014F06ABB28816AAF03D0060E40EC14F072
:104C400073BB288373AF03D0070E40EC14F07CBB1A
:104C500028857CAF03D0080E40EC14F085BB288774
:104C600085AF03D0090E40EC14F08EBB28898EAFBF
:104C700003D00A0E40EC14F097BB288B97AF03D0FB
:104C80000B0E40EC14F04AC042F022514B24436E0C
:104C9000D8B0422A0A0E435ED8A042065FD034BD87
:104CA000258134AF03D0000E40EC14F03DBD2583C8
:104CB0003DAF03D0010E40EC14F046BD258546AF54
:104CC00003D0020E40EC14F04FBD25874FAF03D048
:104CD000030E40EC14F058BD258958AF03D0040EE4
:104CE00040EC14F061BD258B61AF03D0050E40ECA4
:104CF00014F06ABD28816AAF03D0060E40EC14F0B0
:104D000073BD288373AF03D0070E40EC14F07CBD55
:104D100028857CAF03D0080E40EC14F085BD2887B1
:104D200085AF03D0090E40EC14F08EBD28898EAFFC
:104D300003D00A0E40EC14F097BD288B97AF03D038
:104D40000B0E40EC14F04AC042F022514B24436E4B
:104D5000D8B0422A0A0E435ED8A04206186A196AE1
:104D60000DC29CFB0EC29DFB0FC29EFB10C29FFB9F
:104D700011C2A0FB12C2A1FB13C2A2FB14C2A3FB6F
:104D800015C2A4FB16C2A5FB17C2A6FB18C2A7FB3F
:104D900019C2A8FB1AC2A9FB1BC2AAFB1CC2ABFB0F
:104DA0001DC2ACFB1EC2ADFB1FC2AEFB20C2AFFBDF
:104DB00021C2B0FB22C2B1FB23C2B2FB24C2B3FBAF
:104DC0000EA42E910EA405D117B982D0D8909D5172
:104DD00034B719269C5134B71826D8B0192AD89060
:104DE0009F513DB719269E513DB71826D8B0192AB4
:104DF000D890A15146B71926A05146B71826D8B069
:104E0000192AD890A3514FB71926A2514FB7182687
:104E1000D8B0192AD890A55158B71926A45158B717
:104E20001826D8B0192AD890A75161B71926A651CB
:104E300061B71826D8B0192AD890A9516AB719268F
:104E4000A8516AB71826D8B0192AD890AB5173B7B1
:104E50001926AA5173B71826D8B0192AD890AD517F
:104E60007CB71926AC517CB71826D8B0192AD8902F
:104E7000AF5185B71926AE5185B71826D8B0192A73
:104E8000D890B1518EB71926B0518EB71826D8B028
:104E9000192AD890B35197B71926B25197B7182647
:104EA000D8B0192A63C71CF000BC5BCD1CF062C7E8
:104EB0001DF000BC5ACD1DF01D50195CD8A088D043
:104EC000D8A404D01C50185CD8A082D02E9181D0D8
:104ED000D8909D5134BF19269C5134BF1826D8B0A4
:104EE000192AD8909F513DBF19269E513DBF1826C3
:104EF000D8B0192AD890A15146BF1926A05146BF53
:104F00001826D8B0192AD890A3514FBF1926A251FC
:104F10004FBF1826D8B0192AD890A55158BF1926C6
:104F2000A45158BF1826D8B0192AD890A75161BFEC
:104F30001926A65161BF1826D8B0192AD890A951B0
:104F40006ABF1926A8516ABF1826D8B0192AD89066
:104F5000AB5173BF1926AA5173BF1826D8B0192AAE
:104F6000D890AD517CBF1926AC517CBF1826D8B063
:104F7000192AD890AF5185BF1926AE5185BF182682
:104F8000D8B0192AD890B1518EBF1926B0518EBF12
:104F90001826D8B0192AD890B35197BF1926B25104
:104FA00097BF1826D8B0192A6BC71CF000BC63CD78
:104FB0001CF06AC71DF000BC62CD1DF01D50195CCD
:104FC000D8A006D0D8A482D71C50185CD8B07ED701
:104FD0002E81186A196A25A106D09D5119269C5167
:104FE0001826D8B0192A25A306D09F5119269E51FC
:104FF0001826D8B0192A25A506D0A1511926A051E6
:105000001826D8B0192A25A706D0A3511926A251CF
:105010001826D8B0192A25A906D0A5511926A451B9
:105020001826D8B0192A25AB06D0A7511926A651A3
:105030001826D8B0192A28A106D0A9511926A85196
:105040001826D8B0192A28A306D0AB511926AA5180
:105050001826D8B0192A28A506D0AD511926AC516A
:105060001826D8B0192A28A706D0AF511926AE5154
:105070001826D8B0192A28A906D0B1511926B0513E
:105080001826D8B0192A28AB06D0B3511926B25128
:105090001826D8B0192A18C036F019C037F031C018
:1050A0001CF032C01DF0276B2A6B1D50195CD8A074
:1050B00008D0D8A4B3EF2DF01C50185CD8B0B3EFD3
:1050C0002DF018501C5ED8A01D0619501D5E17B992
:1050D000B2D225A134A301D0278125A33DA301D0BD
:1050E000278325A546A301D0278525A74FA301D057
:1050F000278725A958A301D0278925AB61A301D013
:10510000278B28A16AA301D02A8128A373A301D0E9
:105110002A8328A57CA301D02A8528A785A301D0AE
:105120002A8728A98EA301D02A8928AB97A301D06A
:105130002A8B4DEC14F01D501B5CD8A008D0D8A4CD
:1051400074EF2DF01C501A5CD8B074EF2DF025A12F
:1051500034A501D0278125A33DA501D0278325A50E
:1051600046A501D0278525A74FA501D0278725A9CA
:1051700058A501D0278925AB61A501D0278B28A18F
:105180006AA501D02A8128A373A501D02A8328A566
:105190007CA501D02A8528A785A501D02A8728A922
:1051A0008EA501D02A8928AB97A501D02A8B4DEC7A
:1051B00014F01D501B5CD8A008D0D8A474EF2DF0BB
:1051C0001C501A5CD8B074EF2DF025A134A701D083
:1051D000278125A33DA701D0278325A546A701D078
:1051E000278525A74FA701D0278725A958A701D034
:1051F000278925AB61A701D0278B28A16AA701D0F9
:105200002A8128A373A701D02A8328A57CA701D0CF
:105210002A8528A785A701D02A8728A98EA701D08B
:105220002A8928AB97A701D02A8B4DEC14F01D508A
:105230001B5CD8A008D0D8A474EF2DF01C501A5CC9
:10524000D8B074EF2DF025A135A101D034BF01D025
:10525000278125A33EA101D03DBF01D0278325A5ED
:1052600047A101D046BF01D0278525A750A101D075
:105270004FBF01D0278725A959A101D058BF01D020
:10528000278925AB62A101D061BF01D0278B28A15E
:105290006BA101D06ABF01D02A8128A374A101D0DB
:1052A00073BF01D02A8328A57DA101D07CBF01D086
:1052B0002A8528A786A101D085BF01D02A8728A9E1
:1052C0008FA101D08EBF01D02A8928AB98A101D02F
:1052D00097BF01D02A8B4DEC14F01D501B5CD8A059
:1052E00008D0D8A474EF2DF01C501A5CD8B074EF1D
:1052F0002DF025A135A301D034BF01D0278125A3EE
:105300003EA301D03DBF01D0278325A547A301D0EF
:1053100046BF01D0278525A750A301D04FBF01D09C
:10532000278725A959A301D058BF01D0278925ABCC
:1053300062A301D061BF01D0278B28A16BA301D04C
:105340006ABF01D02A8128A374A301D073BF01D002
:105350002A8328A57DA301D07CBF01D02A8528A758
:1053600086A301D085BF01D02A8728A98FA301D0A9
:105370008EBF01D02A8928AB98A301D097BF01D056
:105380002A8B4DEC14F01D501B5CD8A008D0D8A47B
:1053900074EF2DF01C501A5CD8B074EF2DF025A1DD
:1053A00035A501D034BF01D0278125A33EA501D06A
:1053B0003DBF01D0278325A547A501D046BF01D019
:1053C000278525A750A501D04FBF01D0278725A944
:1053D00059A501D058BF01D0278925AB62A501D0BE
:1053E00061BF01D0278B28A16BA501D06ABF01D076
:1053F0002A8128A374A501D073BF01D02A8328A5D0
:105400007DA501D07CBF01D02A8528A786A501D023
:1054100085BF01D02A8728A98FA501D08EBF01D0D2
:105420002A8928AB98A501D097BF01D02A8B4DECD3
:1054300014F01D501B5CD8A008D0D8A474EF2DF038
:105440001C501A5CD8B074EF2DF025A126A101D014
:1054500034BF01D0278125A326A301D03DBF01D0B1
:10546000278325A526A501D046BF01D0278525A7DE
:1054700026A701D04FBF01D0278725A926A901D093
:1054800058BF01D0278925AB26AB01D061BF01D021
:10549000278B28A129A101D06ABF01D02A8128A386
:1054A00029A301D073BF01D02A8328A529A501D043
:1054B0007CBF01D02A8528A729A701D085BF01D0AC
:1054C0002A8728A929A901D08EBF01D02A8928AB13
:1054D00029AB01D097BF01D02A8B4DEC14F01D50A1
:1054E0001B5CD8A006D0D8A4FFD21C501A5CD8B040
:1054F000FBD225A134BF01D025A001D0278125A34F
:105500003DBF01D025A201D0278325A546BF01D0EC
:1055100025A401D0278525A74FBF01D025A601D0FE
:10552000278725A958BF01D025A801D0278925ABF9
:1055300061BF01D025AA01D0278B28A16ABF01D065
:1055400026A001D02A8128A373BF01D026A201D0B2
:105550002A8328A57CBF01D026A401D02A8528A7AC
:1055600085BF01D026A601D02A8728A98EBF01D0E9
:1055700026A801D02A8928AB97BF01D026AA01D03E
:105580002A8B4DEC14F01D501B5CD8A006D0D8A47B
:10559000ABD21C501A5CD8B0A7D225A127B101D03C
:1055A00025A001D043D025A327B301D025A201D047
:1055B0003DD025A527B501D025A401D037D025A7FA
:1055C00027B701D025A601D031D025A927B901D010
:1055D00025A801D02BD025AB27BB01D025AA01D00F
:1055E00025D028A12AB101D026A001D01FD028A300
:1055F0002AB301D026A201D019D028A52AB501D0FE
:1056000026A401D013D028A72AB701D026A601D0FE
:105610000DD028A92AB901D026A801D007D028ABDF
:105620002ABB01D026AA01D001D096D2020E426E2A
:10563000CB0E436E91D225A134AB01D0278125A397
:105640003DAB01D0278325A546AB01D0278525A7F3
:105650004FAB01D0278725A958AB01D0278925ABAF
:1056600061AB01D0278B28A16AAB01D02A8128A386
:1056700073AB01D02A8328A57CAB01D02A8528A74B
:1056800085AB01D02A8728A98EAB01D02A8928AB07
:1056900097AB01D02A8B4DEC14F01D501B5CD8A0A9
:1056A00006D0D8A421D21C501A5CD8B01DD225A196
:1056B00034AD01D0278125A33DAD01D0278325A599
:1056C00046AD01D0278525A74FAD01D0278725A955
:1056D00058AD01D0278925AB61AD01D0278B28A11A
:1056E0006AAD01D02A8128A373AD01D02A8328A5F1
:1056F0007CAD01D02A8528A785AD01D02A8728A9AD
:105700008EAD01D02A8928AB97AD01D02A8B4DEC04
:1057100014F01D501B5CD8A006D0D8A4E5D11C50B5
:105720001A5CD8B0E1D125A134AF01D0278125A3DF
:105730003DAF01D0278325A546AF01D0278525A7FA
:105740004FAF01D0278725A958AF01D0278925ABB6
:1057500061AF01D0278B28A16AAF01D02A8128A38D
:1057600073AF01D02A8328A57CAF01D02A8528A752
:1057700085AF01D02A8728A98EAF01D02A8928AB0E
:1057800097AF01D02A8B4DEC14F01D501B5CD8A0B4
:1057900006D0D8A4A9D11C501A5CD8B0A5D125A197
:1057A00035A701D034B701D0278125A33EA701D06A
:1057B0003DB701D0278325A547A701D046B701D023
:1057C000278525A750A701D04FB701D0278725A946
:1057D00059A701D058B701D0278925AB62A701D0BE
:1057E00061B701D0278B28A16BA701D06AB701D080
:1057F0002A8128A374A701D073B701D02A8328A5D2
:105800007DA701D07CB701D02A8528A786A701D023
:1058100085B701D02A8728A98FA701D08EB701D0DC
:105820002A8928AB98A701D097B701D02A8B4DECD5
:1058300014F01D501B5CD8A006D0D8A455D11C5024
:105840001A5CD8B051D125A135A901D034B701D007
:10585000278125A33EA901D03DB701D0278325A5E7
:1058600047A901D046B701D0278525A750A901D067
:105870004FB701D0278725A959A901D058B701D022
:10588000278925AB62A901D061B701D0278B28A158
:105890006BA901D06AB701D02A8128A374A901D0CD
:1058A00073B701D02A8328A57DA901D07CB701D088
:1058B0002A8528A786A901D085B701D02A8728A9DB
:1058C0008FA901D08EB701D02A8928AB98A901D021
:1058D00097B701D02A8B4DEC14F01D501B5CD8A05B
:1058E00006D0D8A401D11C501A5CD8B0FDD025A197
:1058F00035AB01D034B701D0278125A33EAB01D011
:105900003DB701D0278325A547AB01D046B701D0CD
:10591000278525A750AB01D04FB701D0278725A9F0
:1059200059AB01D058B701D0278925AB62AB01D064
:1059300061B701D0278B28A16BAB01D06AB701D02A
:105940002A8128A374AB01D073B701D02A8328A57C
:105950007DAB01D07CB701D02A8528A786AB01D0CA
:1059600085B701D02A8728A98FAB01D08EB701D087
:105970002A8928AB98AB01D097B701D02A8B4DEC80
:1059800014F01D501B5CD8A006D0D8A4ADD01C507C
:105990001A5CD8B0A9D025A126A101D034B701D076
:1059A000278125A326A301D03DB701D0278325A5B4
:1059B00026A501D046B701D0278525A726A701D067
:1059C0004FB701D0278725A926A901D058B701D004
:1059D000278925AB26AB01D061B701D0278B28A141
:1059E00029A101D06AB701D02A8128A329A301D017
:1059F00073B701D02A8328A529A501D07CB701D08F
:105A00002A8528A729A701D085B701D02A8728A9E8
:105A100029A901D08EB701D02A8928AB29AB01D0A2
:105A200097B701D02A8B4DEC14F01D501B5CD8A009
:105A300006D0D8A459D01C501A5CD8B055D025A196
:105A400034B701D025A001D0278125A33DB701D0CF
:105A500025A201D0278325A546B701D025A401D0D2
:105A6000278525A74FB701D025A601D0278725A9CF
:105A700058B701D025A801D0278925AB61B701D03F
:105A800025AA01D0278B28A16AB701D026A001D072
:105A90002A8128A373B701D026A201D02A8328A582
:105AA0007CB701D026A401D02A8528A785B701D0CC
:105AB00026A601D02A8728A98EB701D026A801D012
:105AC0002A8928AB97B701D026AA01D02A8B4DECA2
:105AD00014F01D501B5CD8A006D0D8A405D01C50D3
:105AE0001A5CD8B001D059D5D8901C361D36D89044
:105AF0001C361D361D501B5CD8A009D0D8A404D07C
:105B00001C501A5CD8A003D0190E246F2CD0D8904A
:105B10001A341E6E1B341F6E1D501F5CD8A009D096
:105B2000D8A404D01C501E5CD8A003D0320E246F21
:105B30001AD01A501E26D8B01F2A1B501F261D50DF
:105B40001F5CD8A009D0D8A404D01C501E5CD8A0DB
:105B500003D04B0E246F07D0640E246F04D0020EC6
:105B6000426ECB0E436E22B02DA10DD0E10EB417C4
:105B7000B517B617B717B817B917BA17BB17BC17A9
:105B8000BD17BE17BF171751D8A43ED036BF258109
:105B90003FBF258348BF258551BF25875ABF25892B
:105BA00063BF258B6CBF288175BF28837EBF288586
:105BB00087BF288790BF288999BF288B2551281136
:105BC000D8B403D0276B2A6B3BD0B4BB2581B5BBBF
:105BD0002583B6BB2585B7BB2587B8BB2589B9BB4F
:105BE000258BBABB2881BBBB2883BCBB2885BDBB2A
:105BF0002887BEBB2889BFBB288B25512811D8B464
:105C00001FD0276B2A6B1CD03050D8B435BA18D0AF
:105C100026B1258126B3258326B5258526B7258778
:105C200026B9258926BB258B29B1288129B328834C
:105C300029B5288529B7288729B9288929BB288B20
:105C4000000EB411B511B611B711B811B911BA11CE
:105C5000BB11BC11BD11BE11BF11186E18B2189046
:105C600018B4189018B6189018B8189018B8189258
:105C700018B8189418B8189618B218A401D0188635
:105C800018B6189218B61894185004A0000E476E53
:105C9000320E186EDCC41AF0DDC41BF017B96DD0DB
:105CA0001850385DD8A025A101D01AA001D038CB5A
:105CB00018F01850415DD8A025A301D01AA201D038
:105CC00041CB18F018504A5DD8A025A501D01AA4E0
:105CD00001D04ACB18F01850535DD8A025A701D0A9
:105CE0001AA601D053CB18F018505C5DD8A025A996
:105CF00001D01AA801D05CCB18F01850655DD8A06F
:105D000025AB01D01AAA01D065CB18F018506E5DF2
:105D1000D8A028A101D01BA001D06ECB18F018503C
:105D2000775DD8A028A301D01BA201D077CB18F0B3
:105D30001850805DD8A028A501D01BA401D080CB2D
:105D400018F01850895DD8A028A701D01BA601D053
:105D500089CB18F01850925DD8A028A901D01BA8B3
:105D600001D092CB18F018509B5DD8A028AB01D081
:105D70001BAA01D09BCB18F06CD01850375DD8B05F
:105D800025A101D01AA001D037CB18F01850405DE2
:105D9000D8B025A301D01AA201D040CB18F01850DA
:105DA000495DD8B025A501D01AA401D049CB18F07F
:105DB0001850525DD8B025A701D01AA601D052CBF9
:105DC00018F018505B5DD8B025A901D01AA801D0F1
:105DD0005BCB18F01850645DD8B025AB01D01AAA7F
:105DE00001D064CB18F018506D5DD8B028A101D057
:105DF0001BA001D06DCB18F01850765DD8B028A349
:105E000001D01BA201D076CB18F018507F5DD8B01E
:105E100028A501D01BA401D07FCB18F01850885DB5
:105E2000D8B028A701D01BA601D088CB18F01850F5
:105E3000915DD8B028A901D01BA801D091CB18F052
:105E400018509A5DD8B028AB01D01BAA01D09ACBCC
:105E500018F01850446E280E4C6E3C0E4D6EFFD05C
:105E60002E91000EEA6E420EE96E040EE26EBB0E3B
:105E700026B82EA801D00FB201D0AB0E26B62EA6A2
:105E800001D00FB201D09B0E26B42EA401D00FB2C8
:105E900001D08B0E26B22EA201D00FB201D07B0E04
:105EA00026B02EA001D00FB201D06B0E25BA2DAABC
:105EB00001D00FB001D05B0E25B82DA801D00FB0D6
:105EC00001D04B0E25B62DA601D00FB001D03B0E50
:105ED00025B42DA401D00FB001D02B0E25B22DA2D8
:105EE00001D00FB001D01B0E25B02DA001D00FB0F6
:105EF00001D00B0EE16E0C0E186EE550EE6E182EF2
:105F0000FCD7010E42BE436E42BE426AE10E2DA195
:105F100004A047163F0E256F286F186A196A0DC234
:105F20009CFB0EC29DFB0FC29EFB10C29FFB11C2C9
:105F3000A0FB12C2A1FB13C2A2FB14C2A3FB15C299
:105F4000A4FB16C2A5FB17C2A6FB18C2A7FB19C269
:105F5000A8FB1AC2A9FB1BC2AAFB1CC2ABFB1DC239
:105F6000ACFB1EC2ADFB1FC2AEFB20C2AFFB21C209
:105F7000B0FB22C2B1FB23C2B2FB24C2B3FB25B0EB
:105F80000FB006D09D5119269C511826D8B0192A59
:105F900025B20FB006D09F5119269E511826D8B0B1
:105FA000192A25B40FB006D0A1511926A0511826E0
:105FB000D8B0192A25B60FB006D0A3511926A25180
:105FC0001826D8B0192A25B80FB006D0A551192621
:105FD000A4511826D8B0192A25BA0FB006D0A75157
:105FE0001926A6511826D8B0192A26B00FB206D005
:105FF000A9511926A8511826D8B0192A26B20FB2CD
:1060000006D0AB511926AA511826D8B0192A26B4A1
:106010000FB206D0AD511926AC511826D8B0192AA6
:1060200026B60FB206D0AF511926AE511826D8B0F9
:10603000192A26B80FB206D0B1511926B051182628
:10604000D8B0192A26BA0FB206D0B3511926B251C8
:106050001826D8B0192A18C036F019C037F0000E2B
:10606000EA6E400EE96E040EE26E6D0E25BA53AA7A
:1060700001D05D0E25B853A801D04D0E25B653A60C
:1060800001D03D0E25B453A401D02D0E25B253A24C
:1060900001D01D0E25B053A001D00D0EE16E020EF1
:1060A000186EE550EE6E182EFCD700BA63D025B1FD
:1060B000279125B3279325B5279525B7279725B988
:1060C000279925BB279B28B12A9128B32A9328B565
:1060D0002A9528B72A9728B92A9928BB2A9B25519F
:1060E0002811D8B442D0276A286A296A2A6A2B6AFA
:1060F0002C6A3A6A3B6A3C6A3D6A3E6A3F6A2451AE
:1061000027B1276E27B3286E27B5296E27B72A6EC9
:1061100027B92B6E27BB2C6E2AB13A6E2AB33B6E81
:106120002AB53C6E2AB73D6E2AB93E6E2ABB3F6E39
:10613000640E25B1276E25B3286E25B5296E25B7C7
:106140002A6E25B92B6E25BB2C6E28B13A6E28B36A
:106150003B6E28B53C6E28B73D6E28B93E6E28BB15
:106160003F6E275125132A51281325CB26FB28CB18
:1061700029FB50D00B0EE06E256B286B2750D8A45E
:1061800025812850D8A425832950D8A425852A50B4
:10619000D8A425872B50D8A425892C50D8A4258B8A
:1061A000000EEA6E400EE96E040EE26E5D0E25B83A
:1061B00053A801D04D0E25B653A601D03D0E25B4EF
:1061C00053A401D02D0E25B253A201D01D0E25B02F
:1061D00053A001D00D0EE16E020E186EE550EE6E6A
:1061E000182EFCD7020EEA6E430EE96E050EE26E23
:1061F0002D0E25B8250E25B61D0E25B4150E25B27B
:106200000D0E25B0050EE16E040E186EE550EE6E13
:10621000182EFCD7030EE06E25CB18F0385018B0BE
:10622000006F18B2026F18B4046F18B6066F18B872
:10623000086F18BA0A6F000E18A0006F18A2026F3C
:1062400018A4046F18A6066F18A8086F18AA0A6F7A
:10625000395018B0016F18B2036F18B4056F18B633
:10626000076F18B8096F18BA0B6F180B18A0016FD9
:1062700018A2036F18A4056F18A6076F18A8096F56
:1062800018AA0B6F020EEA6E430EE96E050EE26E5F
:10629000350E25BA2D0E25B8250E25B61D0E25B4B2
:1062A000150E25B20D0E25B0050EE16E040E186E0A
:1062B000E550EE6E182EFCD7020EE06E0EBE1DD01D
:1062C00004BE04BC1AD0640E276E286E296E2A6E96
:1062D0002B6E2C6E3A6E3B6E3C6E3D6E3E6E3F6E8C
:1062E000A06FA16FA26FA36FA46FA56FA66FA76F1A
:1062F000A86FA96FAA6FAB6F048CD8900C31616F37
:106300000B31606FD890613360330B6A5451551173
:10631000D8A437D00C902750625DD8B432D0D8A022
:106320001ED0626F0C902750D8B421D060C254F2B6
:1063300061C255F2280E625DD8A01DD0605154276D
:10634000D8B0552B61515527410E625DD8A013D0AE
:1063500060515427D8B0552B615155270CD062514C
:10636000275C626F0C80640E275CD8A0DFD70BC25D
:1063700054F20CC255F22750626FD8A44081D8B4B1
:10638000409154515511D8A40B8056515711D8A49F
:1063900037D00C922850635DD8B432D0D8A01ED02C
:1063A000636F0C922850D8B421D060C256F261C2FB
:1063B00057F2280E635DD8A01DD060515627D8B083
:1063C000572B61515727410E635DD8A013D0605100
:1063D0005627D8B0572B615157270CD06351285CF2
:1063E000636F0C82640E285CD8A0DFD70BC256F214
:1063F0000CC257F22850636FD8A44083D8B440939E
:1064000056515711D8A40B8258515911D8A437D0DE
:106410000C942950645DD8B432D0D8A01ED0646FDB
:106420000C942950D8B421D060C258F261C259F2FC
:10643000280E645DD8A01DD060515827D8B0592BC4
:1064400061515927410E645DD8A013D0605158277F
:10645000D8B0592B615159270CD06451295C646F15
:106460000C84640E295CD8A0DFD70BC258F20CC292
:1064700059F22950646FD8A44085D8B4409558513A
:106480005911D8A40B845A515B11D8A437D00C965B
:106490002A50655DD8B432D0D8A01ED0656F0C9656
:1064A0002A50D8B421D060C25AF261C25BF2280EE1
:1064B000655DD8A01DD060515A27D8B05B2B6151C3
:1064C0005B27410E655DD8A013D060515A27D8B024
:1064D0005B2B61515B270CD065512A5C656F0C8684
:1064E000640E2A5CD8A0DFD70BC25AF20CC25BF252
:1064F0002A50656FD8A44087D8B440975A515B1191
:10650000D8A40B865C515D11D8A437D00C982B50C1
:10651000665DD8B432D0D8A01ED0666F0C982B50D0
:10652000D8B421D060C25CF261C25DF2280E665D13
:10653000D8A01DD060515C27D8B05D2B61515D277C
:10654000410E665DD8A013D060515C27D8B05D2B9A
:1065500061515D270CD066512B5C666F0C88640E10
:106560002B5CD8A0DFD70BC25CF20CC25DF22B50C3
:10657000666FD8A44089D8B440995C515D11D8A405
:106580000B885E515F11D8A437D00C9A2C50675DF0
:10659000D8B432D0D8A01ED0676F0C9A2C50D8B483
:1065A00021D060C25EF261C25FF2280E675DD8A0A2
:1065B0001DD060515E27D8B05F2B61515F27410E1F
:1065C000675DD8A013D060515E27D8B05F2B6151B2
:1065D0005F270CD067512C5C676F0C8A640E2C5CB3
:1065E000D8A0DFD70BC25EF20CC25FF22C50676FEF
:1065F000D8A4408BD8B4409B5E515F11D8A40B8ABD
:106600004AD00B6A0C6A2750D8A404D040910AA340
:106610000B8005D040810AA302D00B800C8028504B
:10662000D8A404D040930AA30B8205D040830AA3C8
:1066300002D00B820C822950D8A404D040950AA322
:106640000B8405D040850AA302D00B840C842A5009
:10665000D8A404D040970AA30B8605D040870AA38C
:1066600002D00B860C862B50D8A404D040990AA3E4
:106670000B8805D040890AA302D00B880C882C50C7
:10668000D8A404D0409B0AA30B8A05D0408B0AA350
:1066900002D00B8A0C8A020EE06E0AC218F0F28158
:1066A000F691F49118AE00BE04D03F0E0F14D8B48A
:1066B00002D0F291F481F293F693F49300B21AD0DF
:1066C0004F6B509F6B6B0EAE0FA001D011D00EBE62
:1066D0000FA201D00DD00FA80FBE0AD00FA00FB28D
:1066E00005D00FA40FB602D00FAA1ED0F2831CD083
:1066F000F4831AD0040E4F5DD8B002D08E9E14D011
:106700008E8E080E50BF640E4F5DD8A00DD050BFC6
:1067100008D06B2BF7516B5DD8B0508F50AF4F6BDB
:1067200003D04F6B509F6B6BF299F499F6993150EF
:106730003210D8A4F28918AE00BE35D00EB033D0D6
:1067400017CB18F0F295F495F69518B0F6850EBEB5
:1067500051A601D0F6850EBE51A401D0F28530506D
:1067600018B0D8B401D034BC01D034BE01D0F28509
:1067700035BAF285F2B5F695F297F497F69718B810
:10678000F6870EBE51A201D0F6870EBE51A001D0F1
:10679000F287305018B8D8B401D034AE01D0F287A7
:1067A000F2B7F6970ED0F295F495F69538A638B86C
:1067B000F28538BAF285F297F497F69738A238B492
:1067C000F287196AF2B71980F6B71982F2B51984FF
:1067D000F6B5198619C052F00A0E50A1320E515D5D
:1067E000D8A01FD0516B50A10AD08E988E928E9651
:1067F0008E94909E909C909A9098509112D00850B0
:10680000D8A48E8820B88E8221B08E8621B28E8444
:1068100021B4908E21B6908C21B8908A21BA9088AC
:106820005081020E525DD8A03AD0526B50A31CD0BA
:10683000F3B18C90F3B38C92F3B58C94F3B78C9640
:10684000F3B98C98F3BB8C9AF4B18F88F4B38E8E25
:10685000F4B58A9AF4B78A98F4B90D90F4BB8C9C7D
:10686000F4BD8C9E50931BD0F3B18C80F3B38C821B
:10687000F3B58C84F3B78C86F3B98C88F3BB8C8A20
:10688000F4B18F98F4B38E9EF4B58A8AF4B78A88EF
:10689000F4B90D80F4BB8C8CF4BD8C8E50830A0E41
:1068A000535DD8A03AD0536B50A51CD0F5B18C9055
:1068B000F5B38C92F5B58C94F5B78C96F5B98C98A8
:1068C000F5BB8C9AF6B18F88F6B38E8EF6B58A9AA0
:1068D000F6B78A98F6B90D90F6BB8C9CF6BD8C9EE7
:1068E00050951BD0F5B18C80F5B38C82F5B58C84B6
:1068F000F5B78C86F5B98C88F5BB8C8AF6B18F9884
:10690000F6B38E9EF6B58A8AF6B78A88F6B90D80F8
:10691000F6BB8C8CF6BD8C8E5085F1B18C80F1B3BA
:106920008C82F1B58C84F1B78C86F1B98C88F1BB7F
:106930008C8AF2B18F98F2B38E9EF2B58A8AF2B742
:106940008A88F2B90D80F2BB8C8CF2BD8C8EF1512D
:10695000F311F511186EF251F411F611196E18A019
:106960008C9018A28C9218A48C9418A68C9618A8B7
:106970008C9818AA8C9A19A08F8819A200B201D0FD
:106980008E8E19A48A9A19A68A9819A80D9019AA08
:106990008C9C19AC8C9E0DB0899E0DA0898E0DB07B
:1069A0008B9A0DA08B8A0BA004D0F381F591F19105
:1069B00012D02750D8A404D0F391F591F1910BD0C7
:1069C000640E275CD8A004D0F391F591F18103D037
:1069D000F391F581F1910BA204D0F383F593F19338
:1069E00012D02850D8A404D0F393F593F1930BD090
:1069F000640E285CD8A004D0F393F593F18303D000
:106A0000F393F583F1930BA404D0F385F595F195F9
:106A100012D02950D8A404D0F395F595F1950BD058
:106A2000640E295CD8A004D0F395F595F18503D0C8
:106A3000F395F585F1950BA604D0F387F597F197BB
:106A400012D02A50D8A404D0F397F597F1970BD021
:106A5000640E2A5CD8A004D0F397F597F18703D091
:106A6000F397F587F1970BA804D0F389F599F1997D
:106A700012D02B50D8A404D0F399F599F1990BD0EA
:106A8000640E2B5CD8A004D0F399F599F18903D05A
:106A9000F399F589F1990BAA04D0F38BF59BF19B3F
:106AA0002DD02C50D8A404D0F39BF59BF19B26D07D
:106AB000640E2C5CD8A004D0F39BF59BF18B1ED008
:106AC000F39BF58BF19B1AD0F36BF56B0BA0F19157
:106AD0000BB0F1810BA2F1930BB2F1830BA4F195F2
:106AE0000BB4F1850BA6F1970BB6F1870BA8F199C2
:106AF0000BB8F1890BAAF19B0BBAF18B67EF16F07B
:106B000000EF00F000FE00FE00FC00FB00FD0100B5
:106B100000FE00FE04E900FE0271027002730272C0
:106B2000027502740277027602790278027B027A99
:106B3000027D027C027F027E028102800283028249
:106B4000028502840287028602890288028B028AF9
:106B5000028C028D028E028F0290029102920293A9
:106B600002940295029602970299029802BF02BE11
:106B70000051024200230022000E000F00300033BB
:106B80000034003500320031003800390B340B3549
:106B90000B3D0B3E0B460B470B4F0B500B580B5945
:106BA0000B610B62060006010602060306040605D9
:106BB0000606060706080609060A060B060C060D59
:106BC000060E00FE06100611061206130614061520
:106BD0000616061706180619061A061B061C061DB9
:106BE000061E00FE06200621062206230624062590
:106BF0000626062706280629062A062B062C062D19
:106C0000062E00FE063006310632063306340635FF
:106C10000636063706380639063A063B063C063D78
:106C2000063E00FE0640064106420643064406456F
:106C30000646064706480649064A064B064C064DD8
:106C4000064E00FE065006510652065306540655DF
:106C50000656065706580659065A065B065C065D38
:106C6000065E00FE0660066106620663066406654F
:106C70000666066706680669066A066B066C066D98
:106C8000066E00FE067006710672067306740675BF
:106C90000676067706780679067A067B067C067DF8
:106CA000067E00FE0680068106820683068406852F
:106CB0000686068706880689068A068B068C068D58
:106CC000068E00FE0690069106920693069406959F
:106CD0000696069706980699069A069B069C069DB8
:106CE000069E00FE06A006A106A206A306A406A50F
:106CF00006A606A706A806A906AA06AB06AC06AD18
:106D000006AE00FE06B006B106B206B306B406B57E
:106D100006B606B706B806B906BA06BB06BC06BD77
:106D200006BE00FE02A002A102A202A302A402A5C6
:106D300002A602A702A802A902AA02AB00FE020450
:106D400000250026040604160426043604460456CC
:106D5000046604760486049604A604B6040904199D
:106D600004290439044904590469047904890499FB
:106D700004A904B9026C026D026E00FE02390237EA
:106D8000023502330096009700980099009A009B04
:106D9000009C009D009E009F00A000A100A200A3F7
:106DA00000A400A500A600A700A800A900AA00ABA7
:106DB00000AC00AD00AE00AF0B6A0B6B0B730B7435
:106DC0000B7C0B7D040B040A040504040403040279
:106DD00004010400041B041A04150414041304120F
:106DE00004110410042B042A04250424042304227F
:106DF00004210420043B043A0435043404330432EF
:106E000004310430044B044A04450444044304425E
:106E100004410440045B045A0455045404530452CE
:106E200004510450046B046A04650464046304623E
:106E300004610460047B047A0475047404730472AE
:106E400004710470048B048A04850484048304821E
:106E500004810480049B049A04950494049304928E
:106E60000491049004AB04AA04A504A404A304A2FE
:106E700004A104A004BB04BA04B504B404B304B26E
:106E800004B104B00B850B860B8E0B8F0B970B9800
:106E900000FE00FE0B2E00FE0037003602430244C7
:106EA0000245024602680269004000410042004378
:106EB000004400FE00FE004700480049004A004B25
:106EC000004C004D00FE00FE00FE00FE00FE00FE35
:106ED00000FE00FE00FE00FE00FE00FE00FE00FEC2
:106EE00000FE00FE00FE00FE00FE00FE00FE00FEB2
:106EF00000FE00FE00FE00FE00FE00FE00FE023A64
:106F000000FE02FE00FF00FF00FF00FF00FF00FF89
:106F100000FF00FF00FF00FF00FF00FF00FF00FF79
:106F200000FF00FF04E900FF00FF00FF02710321E2
:106F300002700320027303230272032202750325E9
:106F400002740324027703270276032602790329B9
:106F500002780328027B032B027A032A027D032D89
:106F6000027C032C027F032F027E032E0281033159
:106F70000280033002830333028203320285033529
:106F800002840334028703370286033602890339F9
:106F900002880338028B033B028A033A028C033CCB
:106FA000028D033D028E033E028F033F0290034099
:106FB0000291034102920342029303430294034469
:106FC00002950345029603460297034700FF00FF20
:106FD00000FF00FF00FF00FF00FF00FF005100FF67
:106FE000024200FF002300FF002200FF000E00FF0E
:106FF000005700FF003000FF003300FF003400FFA7
:10700000003500FF003200FF003100FF003800FFB4
:10701000003900FF00FF00FF00FF00FF00FF00FF3E
:1070200000FF00FF00FF00FF00FF00FF00FF00FF68
:1070300000FF00FF00FF00FF00FF00FF00FF00FF58
:1070400000FF00FF0600035106010352060203532E
:1070500006030354060403550605035606060357A4
:1070600006070358060803590609035A060A035B74
:10707000060B035C060C035D060D035E060E035F44
:1070800000FF00FF06100360061103610612036291
:1070900006130363061403640615036506160366E8
:1070A000061703670618036806190369061A036AB8
:1070B000061B036B061C036C061D036D061E036E88
:1070C00000FF00FF0620036F0621037006220371F4
:1070D000062303720624037306250374062603752C
:1070E000062703760628037706290378062A0379FC
:1070F000062B037A062C037B062D037C062E037DCC
:1071000000FF00FF063003A0063103A1063203A2F0
:10711000063303A3063403A4063503A5063603A6E7
:10712000063703A7063803A8063903A9063A03AAB7
:10713000063B03AB063C03AC063D03AD063E03AE87
:1071400000FF00FF064003AF064103B0064203B153
:10715000064303B2064403B3064503B4064603B52B
:10716000064703B6064803B7064903B8064A03B9FB
:10717000064B03BA064C03BB064D03BC064E03BDCB
:1071800000FF00FF065003BE065103BF065203C0B6
:10719000065303C1065403C2065503C3065603C46F
:1071A000065703C5065803C6065903C7065A03C83F
:1071B000065B03C9065C03CA065D03CB065E03CC0F
:1071C00000FF00FF066003CD066103CE066203CF19
:1071D000066303D0066403D1066503D2066603D3B3
:1071E000066703D4066803D5066903D6066A03D783
:1071F000066B03D8066C03D9066D03DA066E03DB53
:1072000000FF00FF067003DC067103DD067203DE7B
:10721000067303DF067403E0067503E1067603E2F6
:10722000067703E3067803E4067903E5067A03E6C6
:10723000067B03E7067C03E8067D03E9067E03EA96
:1072400000FF00FF068003EB068103EC068203EDDE
:10725000068303EE068403EF068503F0068603F13A
:10726000068703F2068803F3068903F4068A03F50A
:10727000068B03F6068C03F7068D03F8068E03F9DA
:1072800000FF00FF06900560069105610692056209
:1072900006930563069405640695056506960566DE
:1072A000069705670698056806990569069A056AAE
:1072B000069B056B069C056C069D056D069E056E7E
:1072C00000FF00FF06A0056F06A1057006A205716C
:1072D00006A3057206A4057306A5057406A6057522
:1072E00006A7057606A8057706A9057806AA0579F2
:1072F00006AB057A06AC057B06AD057C06AE057DC2
:1073000000FF00FF06B0057E06B1057F06B20580CE
:1073100006B3058106B4058206B5058306B6058465
:1073200006B7058506B8058606B9058706BA058835
:1073300006BB058906BC058A06BD058B06BE058C05
:1073400000FF00FF02A000FF02A100FF02A200FF59
:1073500002A300FF02A400FF02A500FF02A600FF97
:1073600002A700FF02A800FF02A900FF02AA00FF77
:1073700002AB00FF00FF00FF00FF00FF00FF00FF67
:1073800000FF00FF00FF00FF00FF00FF00FF00FF05
:1073900000FF00FF00FF00FF00FF00FF00FF00FFF5
:1073A00000FF00FF00FF00FF00FF00FF00FF00FFE5
:1073B00000FF00FF00FF00FF00FF00FF00FF00FFD5
:1073C00000FF00FF00FF00FF00FF00FF00FF00FFC5
:1073D00000FF00FF00FF00FF00FF00FF00FF00FFB5
:1073E00000FF00FF029C058F029D0590029E059103
:1073F00000FF00FF023903500237034F0235034EEE
:107400000233034D009600FF009700FF009800FF35
:10741000009900FF009A00FF009B00FF009C00FF06
:10742000009D00FF009E00FF009F00FF00A000FFE6
:1074300000A100FF00A200FF00A300FF00A400FFC6
:1074400000A500FF00A600FF00A700FF00A800FFA6
:1074500000A900FF00AA00FF00AB00FF00AC00FF86
:1074600000AD00FF00AE00FF00AF00FF00FF00FF17
:1074700000FF00FF00FF00FF00FF00FF00FF00FF14
:1074800000FF00FF00FF00FF00FF00FF00FF00FF04
:1074900000FF00FF00FF00FF00FF00FF00FF00FFF4
:1074A00000FF00FF00FF00FF00FF00FF00FF00FFE4
:1076800000FF00FF01C600FF01C700FF01C800FFA7
:1076900001C900FF038000FF038100FF038200FF98
:1076A000038300FF038400FF038500FF038600FFC0
:1076B000038700FF038800FF038900FF038A00FFA0
:1076C000038B00FF038C00FF038D00FF038E00FF80
:1076D000038F00FF039000FF039100FF039200FF60
:1076E000039300FF039400FF039500FF00FF00FFDA
:1076F00000FF00FF00FF00FF023A034C00FF00FF05
:1077000000FF00FF700B0151700B0C51700B1751F3
:10771000700B2251700B2D51700B3851700B43516F
:10772000700B4E51700B5951700B6451700B6F51AF
:10773000700B7A51700B85517006905170089651FC
:10774000700BAD51700BB851700BC351700BCE5113
:10775000700AD9517005E4517007E951600B01516D
:1077600060010C51600B0F51600B1A51600B2551D9
:10777000600B3051600B3B51600A4651600652511C
:10778000600259516006A0516006A6516006E051A2
:10779000600AE951600B6051600B6B51600B7651D0
:1077A000600B8151600B8C51600897516004AD51A2
:1077B000600B6052600B6B52600B7652600B815213
:1077C000600B8C52600897526004AD52600B60539E
:1077D000600B6B53600B7653600B8153600B8C53C3
:1077E000600897536004AD53600B6054600B6B549A
:1077F000600B7654600B8154600B8C546008975476
:107800006004AD54600B6055600B6B55600B765592
:10781000600B8155600B8C55600897556004AD5521
:107820003F0601513F0B08513F0B13513F0B1E51B7
:107830003F0B29513F0B34513F0B3F513F0B4A51F6
:107840003F0B55513F0BD8513F02EF513F02F451CE
:107850003F0B60513F0B6B513F0B76513F0B8151FA
:107860003F0B8C513F0B97513F0BA2513F0BAD513A
:107870003F0BB8513F0BC3513F0ACE513F06E35176
:107880003F06E9513F03F1513F0360563F037F56E6
:107890003F039E563F03BD563F03DC563006015161
:1078A000300B0851300B1351300B1E51300B295146
:1078B000300B3451300B3F51300B4A51300B555186
:1078C000300BD8513002EF513002F451300B60517F
:1078D000300B6B51300B7651300B8151300B8C518A
:1078E000300B9751300BA251300BAD51300BB851CA
:1078F000300BC351300ACE513006E3513006E95106
:107900003003F1513003605630037F5630039E56EA
:107910003003DB563003DC5650050151500513513E
:107920005009225150024E515004EC512006015191
:10793000200B0851200B135120061E51200B2851FB
:10794000200B3351200B3E512007495120025A5140
:10795000B0040151B0030651B0030B51B0030F51F5
:10796000B1040151B1030651B1030B51B1030F51E1
:10797000B2040151B2030651B2030B51B2030F51CD
:10798000B3040151B3030651B3030B51B3030F51B9
:10799000B4040151B4030651B4030B51B4030F51A5
:1079A000B5040151B5030651B5030B51B5030F5191
:1079B000B6040151B6030651B6030B51B6030F517D
:1079C000B7040151B7030651B7030B51B7030F5169
:1079D000B8040151B8030651B8030B51B8030F5155
:1079E000B9040151B9030651B9030B51B9030F5141
:1079F000BA040151BA030651BA030B51BA030F512D
:107A0000BB040151BB030651BB030B51BB030F5118
:107A1000A0000000A0000000A0000000A0000000E6
:107A2000A0000000A0000000A0000000A0000000D6
:107A3000A0000000A0000000A1000000A1000000C4
:107A4000A1000000A1000000A1000000A1000000B2
:107A5000A1000000A1000000A1000000A1000000A2
:107A60000000000000000000000000000000000016
:107A70000000000000000000000000000000000006
:107A80000000000001A401A501A601A7008000815B
:107A900000820083008400850086008700880089BA
:107AA000008A008B008C008D008E008F009000916A
:107AB000009200930094009500FF00FF00FF00FF7C
:107AC00000FF00FF00FE00FE07000701070207039A
:107AD000070407050706070707080709070A070B32
:107AE000070C070D070E070F0710071107120713E2
:107AF000071407150716071700FE00FE00FE00FE1C
:107B000007180719071A071B071C071D071E071F61
:107B10000720072107220723072407250726072711
:107B200007280729072A072B072C072D072E072FC1
:107B30000730073107320733073407350736073771
:107B400007380739073A073B073C073D073E073F21
:107B500007400741074207430744074507460747D1
:107B600007480749074A074B074C074D074E074F81
:107B70000750075107520753075407550756075731
:107B800007580759075A075B075C075D075E075FE1
:107B90000760076107620763076407650766076791
:107BA00007680769076A076B076C076D076E076F41
:107BB00007700771077207730774077507760777F1
:107BC00007780779077A077B077C077D077E077FA1
:107BD0000780078107820783078407850786078751
:107BE00007880789078A078B078C078D078E078F01
:107BF00007900791079207930794079507960797B1
:107C00000798079900FE00FE00FE00FE079A079BFA
:107C1000079C079D079E079F07A007A107A207A330
:107C200007A407A500FE00FE07A607A707A807A947
:107C300000FE00FE00FE00FE00FE00FE00FE00FE54
:107C400000FE00FE07DE07DF07E007E107E207E3CB
:107C500007E407E507E607E707E807E907EA07EBB0
:107C600007EC07ED07EE07EF07F007F107F207F360
:107C700007F407F507F607F707F807F907FA07FB10
:107C800007FC07FD07FE07FF0800080108020803BC
:107C9000080408050806080708080809080A080B68
:107CA000080C080D080E080F081008110812081318
:107CB000081408150816081708180819081A081BC8
:107CC000081C081D081E081F082008210822082378
:107CD000082408250826082708280829082A082B28
:107CE000082C082D082E082F0830083108320833D8
:107CF000083408350836083708380839083A083B88
:107D0000083C083D083E083F084008410842084337
:107D1000084408450846084708480849084A084BE7
:107D2000084C084D084E084F085008510852085397
:107D3000085408550856085708580859085A085B47
:107D400000FE00FE07AA07AB07AC07AD07AE07AF02
:107D500007B007B107B207B307B407B507B607B74F
:107D600007B807B907BA07BB07BC07BD07BE07BFFF
:107D700007C007C100FE00FE085C085D085E085FE2
:107D8000086008610862086300FE00FE00FE00FE55
:107D900000FE00FE00FE00FE00FE00FE00FE00FEF3
:107DA00000FE00FE00FE00FE00FE00FE00FE00FEE3
:107DB00000FE00FE00FE00FE00FE00FE00FE00FED3
:107DC00000FE00FE00FE00FE00FE00FE00FE00FEC3
:107DD00000FE00FE00FE00FE00FE00FE00FE00FEB3
:107DE00000FE00FE00FE00FE00FE00FE00FE00FEA3
:107DF00000FE00FE00FE00FE00FE00FE00FE00FE93
:107E000000FE00FE00FE00FE00FE00FE00FE00FE82
:107E100000FE00FE00FE00FE00FE00FE00FE00FE72
:107E200000FE00FE00FE00FE00FE00FE00FE00FE62
:107E300000FE00FE00FE00FE00FE00FE00FE00FE52
:107E400000FE00FE07C207C307C407C507C607C771
:107E500007C807C907CA07CB07CC07CD00FE00FE3D
:107E600000FE00FE00FE00FE07CE07CF07D007D1C0
:107E700007D207D307D407D507D607D707D807D91E
:107E800007DA07DB07DC07DD0AB00AB10AB20AB37A
:107E900000FE00FE00FE00FE00FE00FE00FE00FEF2
:107EA00000FE00FE00FE00FE00FE00FE00FE00FEE2
:107EB00000FE00FE00FE00FE00FE00FE00FE00FED2
:107EC00000FE00FE00FE00FE00FE00FE00FE00FEC2
:107ED00000FE00FE00FE00FE00FE00FE00FE00FEB2
:107EE00000FE00FE00FE00FE00FE00FE00FE00FEA2
:107EF00000FE00FE00FE00FE00FE00FE00FE00FE92
:107F000000FE00FE00FE00FE00FE00FE00FE00FE81
:107F100000FE00FE00FE00FE00FE00FE00FE00FE71
:107F200000FE00FE00FE00FE00FE00FE00FE00FE61
:107F300000FE00FE00FE00FE00FE00FE00FE00FE51
:107F400000FE00FE00FE00FE00FE00FE00FE00FE41
:107F500000FE00FE00FE00FE00FE00FE00FE00FE31
:107F600000FE00FE00FE00FE00FE00FE00FE00FE21
:107F700000FE00FE00FE00FE00FE00FE00FE00FE11
:107F800000FE00FE00FE00FE00FE00FE00FE00FE01
:107F900000FE00FE00FE00FE00FE00FE00FE00FEF1
:107FA00000FE00FE00FE00FE00FE00FE00FE00FEE1
:107FB00000FE00FE00FE00FE00FE00FE00FE00FED1
:107FC00000FE00FE00FE00FE00FE00FE00FE00FEC1
:107FD00000FE00FE00FE00FE00FE00FE00FE00FEB1
:107FE00000FE00FE00FE00FE00FE00FE00FE00FEA1
:107FF00000FE00FE00FE00FE00FE00FE00FE00FE91
:1080000000FE00FE00FE00FE00FE00FE00FE00FE80
:1080100000FE00FE00FE00FE00FE00FE00FE00FE70
:1080200000FE00FE00FE00FE00FE00FE00FE00FE60
:1080300000FE00FE00FE00FE00FE00FE00FE00FE50
:1080400000FE00FE0864086508660867086808699D
:10805000086A086B086C086D086E086F0870087174
:108060000872087308740875087608770878087924
:10807000087A087B087C087D087E087F08800881D4
:108080000882088308840885088608870888088984
:10809000088A088B088C088D088E088F0890089134
:1080A00008920893089408950896089708980899E4
:1080B000089A089B089C089D089E089F08A008A194
:1080C00008A208A308A408A508A608A708A808A944
:1080D00008AA08AB08AC08AD08AE08AF08B008B1F4
:1080E00008B208B308B408B508B608B708B808B9A4
:1080F00008BA08BB08BC08BD08BE08BF08C008C154
:1081000008C208C308C408C508C608C708C808C903
:1081100008CA08CB08CC08CD08CE08CF08D008D1B3
:1081200008D208D308D408D508D608D708D808D963
:1081300008DA08DB08DC08DD08DE08DF08E008E113
:1081400000FE00FE00FE00FE00FE00FE00FE00FE3F
:1081500000FE00FE00FE00FE00FE00FE00FE00FE2F
:1081600000FE00FE00FE00FE00FE00FE00FE00FE1F
:1081700000FE00FE00FE00FE08E208E308E408E559
:1081800008E608E708E808E900FE00FE00FE00FE39
:1081900000FE00FE00FE00FE00FE00FE00FE00FEEF
:1081A00000FE00FE00FE00FE00FE00FE00FE00FEDF
:1081B00000FE00FE00FE00FE00FE00FE00FE00FECF
:1081C00000FE00FE00FE00FE00FE00FE00FE00FEBF
:1081D00000FE00FE00FE00FE00FE00FE00FE00FEAF
:1081E00000FE00FE00FE00FE00FE00FE00FE00FE9F
:1081F00000FE00FE00FE00FE00FE00FE00FE00FE8F
:1082000000FE00FE00FE00FE00FE00FE00FE00FE7E
:1082100000FE00FE00FE00FE00FE00FE00FE00FE6E
:1082200000FE00FE00FE00FE00FE00FE00FE00FE5E
:1082300000FE00FE00FE00FE00FE00FE00FE00FE4E
:1082400000FE00FE08EA08EB08EC08ED08EE08EF77
:1082500008F008F108F208F308F408F508F608F742
:1082600008F808F908FA08FB08FC08FD08FE08FFF2
:10827000090009010902090309040905090609079A
:1082800009080909090A090B090C090D090E090F4A
:1082900009100911091209130914091509160917FA
:1082A00009180919091A091B091C091D091E091FAA
:1082B000092009210922092309240925092609275A
:1082C00009280929092A092B092C092D092E092F0A
:1082D00009300931093209330934093509360937BA
:1082E00009380939093A093B093C093D093E093F6A
:1082F000094009410942094309440945094609471A
:1083000009480949094A094B094C094D094E094FC9
:108310000950095109520953095409550956095779
:1083200009580959095A095B095C095D095E095F29
:1083300009600961096209630964096509660967D9
:1083400000FE00FE00FE00FE00FE00FE00FE00FE3D
:1083500000FE00FE00FE00FE00FE00FE00FE00FE2D
:1083600000FE00FE00FE00FE00FE00FE00FE00FE1D
:1083700000FE00FE00FE00FE09680969096A096B3B
:10838000096C096D096E096F00FE00FE00FE00FE1B
:1083900000FE00FE00FE00FE00FE00FE00FE00FEED
:1083A00000FE00FE00FE00FE00FE00FE00FE00FEDD
:1083B00000FE00FE00FE00FE00FE00FE00FE00FECD
:1083C00000FE00FE00FE00FE00FE00FE00FE00FEBD
:1083D00000FE00FE00FE00FE00FE00FE00FE00FEAD
:1083E00000FE00FE00FE00FE00FE00FE00FE00FE9D
:1083F00000FE00FE00FE00FE00FE00FE00FE00FE8D
:1084000000FE00FE00FE00FE00FE00FE00FE00FE7C
:1084100000FE00FE00FE00FE00FE00FE00FE00FE6C
:1084200000FE00FE00FE00FE00FE00FE00FE00FE5C
:1084300000FE00FE00FE00FE00FE00FE00FE00FE4C
:1084400000FE00FE0970097109720973097409754B
:108450000976097709780979097A097B097C097D08
:10846000097E097F098009810982098309840985B8
:108470000986098709880989098A098B098C098D68
:10848000098E098F09900991099209930994099518
:108490000996099709980999099A099B099C099DC8
:1084A000099E099F09A009A109A209A309A409A578
:1084B00009A609A709A809A909AA09AB09AC09AD28
:1084C00009AE09AF09B009B109B209B309B409B5D8
:1084D00009B609B709B809B909BA09BB09BC09BD88
:1084E00009BE09BF09C009C109C209C309C409C538
:1084F00009C609C709C809C909CA09CB09CC09CDE8
:1085000009CE09CF09D009D109D209D309D409D597
:1085100009D609D709D809D909DA09DB09DC09DD47
:1085200009DE09DF09E009E109E209E309E409E5F7
:1085300009E609E709E809E909EA09EB09EC09EDA7
:1085400000FE00FE00FE00FE00FE00FE00FE00FE3B
:1085500000FE00FE00FE00FE00FE00FE00FE00FE2B
:1085600000FE00FE00FE00FE00FE00FE00FE00FE1B
:1085700000FE00FE00FE00FE09EE09EF09F009F121
:1085800009F209F309F409F500FE00FE00FE00FE01
:1085900000FE00FE00FE00FE00FE00FE00FE00FEEB
:1085A00000FE00FE00FE00FE00FE00FE00FE00FEDB
:1085B00000FE00FE00FE00FE00FE00FE00FE00FECB
:1085C00000FE00FE00FE00FE00FE00FE00FE00FEBB
:1085D00000FE00FE00FE00FE00FE00FE00FE00FEAB
:1085E00000FE00FE00FE00FE00FE00FE00FE00FE9B
:1085F00000FE00FE00FE00FE00FE00FE00FE00FE8B
:1086000000FE00FE00FE00FE00FE00FE00FE00FE7A
:1086100000FE00FE00FE00FE00FE00FE00FE00FE6A
:1086200000FE00FE00FE00FE00FE00FE00FE00FE5A
:1086300000FE00FE00FE00FE00FE00FE00FE00FE4A
:1086400000FE00FE09F609F709F809F909FA09FB25
:1086500009FC09FD09FE09FF0A000A010A020A03D2
:108660000A040A050A060A070A080A090A0A0A0B7E
:108670000A0C0A0D0A0E0A0F0A100A110A120A132E
:108680000A140A150A160A170A180A190A1A0A1BDE
:108690000A1C0A1D0A1E0A1F0A200A210A220A238E
:1086A0000A240A250A260A270A280A290A2A0A2B3E
:1086B0000A2C0A2D0A2E0A2F0A300A310A320A33EE
:1086C0000A340A350A360A370A380A390A3A0A3B9E
:1086D0000A3C0A3D0A3E0A3F0A400A410A420A434E
:1086E0000A440A450A460A470A480A490A4A0A4BFE
:1086F0000A4C0A4D0A4E0A4F0A500A510A520A53AE
:108700000A540A550A560A570A580A590A5A0A5B5D
:108710000A5C0A5D0A5E0A5F0A600A610A620A630D
:108720000A640A650A660A670A680A690A6A0A6BBD
:108730000A6C0A6D0A6E0A6F0A700A710A720A736D
:1087400000FE00FE00FE00FE00FE00FE00FE00FE39
:1087500000FE00FE00FE00FE00FE00FE00FE00FE29
:1087600000FE00FE00FE00FE00FE00FE00FE00FE19
:1087700000FE00FE00FE00FE0A740A750A760A7703
:108780000A780A790A7A0A7B00FE00FE00FE00FEE3
:1087900000FE00FE00FE00FE00FE00FE00FE00FEE9
:1087A00000FE00FE00FE00FE00FE00FE00FE00FED9
:1087B00000FE00FE00FE00FE00FE00FE00FE00FEC9
:1087C00000FE00FE00FE00FE00FE00FE00FE00FEB9
:1087D00000FE00FE00FE00FE00FE00FE00FE00FEA9
:1087E00000FE00FE00FE00FE00FE00FE00FE00FE99
:1087F00000FE00FE00FE00FE00FE00FE00FE00FE89
:1088000000FE00FE00FE00FE00FE00FE00FE00FE78
:1088100000FE00FE00FE00FE00FE00FE00FE00FE68
:1088200000FE00FE00FE00FE00FE00FE00FE00FE58
:1088300000FE00FE00FE00FE00FE00FE00FE00FE48
:1088400000FE00FE00FE00FE07000701070207030E
:10885000070407050706070707080709070A070BA4
:1088600000FE00FE070C070D070E070F071007118B
:108870000712071307140715071607170718071914
:10888000071A071B071C071D071E071F07200721C4
:108890000722072307240725072607270728072974
:1088A000072A072B072C072D072E072F0730073124
:1088B00007320733073407350736073707380739D4
:1088C000073A073B073C073D073E073F0740074184
:1088D0000742074307440745074607470748074934
:1088E000074A074B074C074D074E074F07500751E4
:1088F0000752075307540755075607570758075994
:10890000075A075B075C075D075E075F0760076143
:1089100007620763076407650766076707680769F3
:10892000076A076B076C076D076E076F07700771A3
:108930000772077307740775077607770778077953
:10894000077A077B077C077D077E077F0780078103
:1089500007820783078407850786078707880789B3
:10896000078A078B078C078D078E078F0790079163
:108970000792079307940795079607970798079913
:10898000079A079B079C079D079E079F07A007A1C3
:1089900007A207A307A407A507A607A707A807A973
:1089A00007AA07AB07AC07AD07AE07AF07B007B123
:1089B00007B207B307B407B507B607B707B807B9D3
:1089C00007BA07BB07BC07BD07BE07BF07C007C183
:1089D00007C207C307C407C507C607C707C807C933
:1089E00007CA07CB07CC07CD07CE07CF07D007D1E3
:1089F00007D207D307D407D507D607D707D807D993
:108A000007DA07CB07DC07DD07DE07DF07E007E152
:108A100007E207E307E407E507E607E707E807E9F2
:108A200007EA07EB07EC07ED07EE07EF07F007F1A2
:108A300007F207F307F407F507F607F707F807F952
:108A400007FA07FB07FC07FD07FE07FF0800080100
:108A500008020803080408050806080708080809AA
:108A6000080A080B080C080D080E080F081008115A
:108A7000081208130814081508160817081808190A
:108A8000081A081B081C081D081E081F08200821BA
:108A9000082208230824082508260827082808296A
:108AA000082A082B082C082D082E082F083008311A
:108AB00008320833083408350836083708380839CA
:108AC000083A083B083C083D083E083F084008417A
:108AD000084208430844084508460847084808492A
:108AE000084A084B084C084D084E084F08500851DA
:108AF000085208530854085508560857085808598A
:108B0000085A085B085C085D085E085F0860086139
:108B100008620863086408650866086708680869E9
:108B2000086A086B086C086D086E086F0870087199
:108B30000872087308740875087608770878087949
:108B4000087A087B087C087D087E087F08800881F9
:108B500008820883088408850886088708880889A9
:108B6000088A088B088C088D088E088F0890089159
:108B70000892089308940895089608970898089909
:108B8000089A089B089C089D089E089F08A008A1B9
:108B900008A208A308A408A508A608A708A808A969
:108BA00008AA08AB08AC08AD08AE08AF08B008B119
:108BB00008B208B308B408B508B608B708B808B9C9
:108BC00008BA08BB08BC08BD08BE08BF08C008C179
:108BD00008C208C308C408C508C608C708C808C929
:108BE00008CA08CB08CC08CD08CE08CF08D008D1D9
:108BF00008D208D308D408D508D608D708D808D989
:108C000008DA08DB08DC08DD08DE08DF08E008E138
:108C100008E208E308E408E508E608E700FE00FECD
:108C200000FE00FE00FE00FE00FE00FE00FE00FE54
:108C300000FE00FE00FE00FE00FE00FE00FE00FE44
:108C400000FE00FE08E808E908EA08EB08EC08ED79
:108C500000FE00FE00FE00FE00FE00FE00FE00FE24
:108C600000FE00FE00FE00FE00FE00FE00FE00FE14
:108C700000FE00FE00FE00FE00FE00FE00FE00FE04
:108C800000FE00FE00FE00FE00FE00FE00FE00FEF4
:108C900000FE00FE00FE00FE00FE00FE00FE00FEE4
:108CA00000FE00FE00FE00FE00FE00FE00FE00FED4
:108CB00000FE00FE00FE00FE00FE00FE00FE00FEC4
:108CC00008EE08EF08F008F108F208F300FE00FED5
:108CD00000FE00FE00FE00FE00FE00FE00FE00FEA4
:108CE00000FE00FE00FE00FE00FE00FE00FE00FE94
:108CF00000FE00FE00FE00FE00FE00FE00FE00FE84
:108D000000FE00FE00FE00FE00FE00FE00FE00FE73
:108D100000FE00FE00FE00FE00FE00FE00FE00FE63
:108D200000FE00FE00FE00FE00FE00FE00FE00FE53
:108D300000FE00FE00FE00FE00FE00FE08F408F546
:108D400008F608F708F808F900FE00FE00FE00FE2D
:108D500000FE00FE00FE00FE00FE00FE00FE00FE23
:108D600000FE00FE00FE00FE00FE00FE00FE00FE13
:108D700000FE00FE00FE00FE00FE00FE00FE00FE03
:108D800000FE00FE00FE00FE00FE00FE00FE00FEF3
:108D900000FE00FE00FE00FE00FE00FE00FE00FEE3
:108DA00000FE00FE00FE00FE00FE00FE00FE00FED3
:108DB00000FE00FE00FE00FE08FA08FB08FC08FDAD
:108DC00008FE08FF00FE00FE00FE00FE00FE00FEA2
:108DD00000FE00FE00FE00FE00FE00FE00FE00FEA3
:108DE00000FE00FE00FE00FE00FE00FE00FE00FE93
:108DF00000FE00FE00FE00FE00FE00FE00FE00FE83
:108E000000FE00FE00FE00FE00FE00FE00FE00FE72
:108E100000FE00FE00FE00FE00FE00FE00FE00FE62
:108E200000FE00FE00FE00FE00FE00FE00FE00FE52
:108E300000FE00FE0AF00AF10AF20AF30AF40AF54B
:108E400000FE00FE00FE00FE090009010902090300
:108E5000090409050906090709080909090A090B8E
:108E600000FE00FE090C090D090E090F0910091179
:108E700009120913091409150916091709180919FE
:108E8000091A091B091C091D091E091F09200921AE
:108E9000092209230924092509260927092809295E
:108EA000092A092B092C092D092E092F093009310E
:108EB00009320933093409350936093709380939BE
:108EC000093A093B093C093D093E093F094009416E
:108ED000094209430944094509460947094809491E
:108EE000094A094B094C094D094E094F09500951CE
:108EF000095209530954095509560957095809597E
:108F0000095A095B095C095D095E095F096009612D
:108F100009620963096409650966096709680969DD
:108F2000096A096B096C096D096E096F097009718D
:108F3000097209730974097509760977097809793D
:108F4000097A097B097C097D097E097F09800981ED
:108F5000098209830984098509860987098809899D
:108F6000098A098B098C098D098E098F099009914D
:108F700009920993099409950996099709980999FD
:108F8000099A099B099C099D099E099F09A009A1AD
:108F900009A209A309A409A509A609A709A809A95D
:108FA00009AA09AB09AC09AD09AE09AF09B009B10D
:108FB00009B209B309B409B509B609B709B809B9BD
:108FC00009BA09BB09BC09BD09BE09BF09C009C16D
:108FD00009C209C309C409C509C609C709C809C91D
:108FE00009CA09CB09CC09CD09CE09CF09D009D1CD
:108FF00009D209D309D409D509D609D709D809D97D
:1090000009DA09CB09DC09DD09DE09DF09E009E13C
:1090100009E209E309E409E509E609E709E809E9DC
:1090200009EA09EB09EC09ED09EE09EF09F009F18C
:1090300009F209F309F409F509F609F709F809F93C
:1090400009FA09FB09FC09FD09FE09FF0C000C01E6
:109050000C020C030C040C050C060C070C080C0984
:109060000C0A0C0B0C0C0C0D0C0E0C0F0C100C1134
:109070000C120C130C140C150C160C170C180C19E4
:109080000C1A0C1B0C1C0C1D0C1E0C1F0C200C2194
:109090000C220C230C240C250C260C270C280C2944
:1090A0000C2A0C2B0C2C0C2D0C2E0C2F0C300C31F4
:1090B0000C320C330C340C350C360C370C380C39A4
:1090C0000C3A0C3B0C3C0C3D0C3E0C3F0C400C4154
:1090D0000C420C430C440C450C460C470C480C4904
:1090E0000C4A0C4B0C4C0C4D0C4E0C4F0C500C51B4
:1090F0000C520C530C540C550C560C570C580C5964
:109100000C5A0C5B0C5C0C5D0C5E0C5F0C600C6113
:109110000C620C630C640C650C660C670C680C69C3
:109120000C6A0C6B0C6C0C6D0C6E0C6F0C700C7173
:109130000C720C730C740C750C760C770C780C7923
:109140000C7A0C7B0C7C0C7D0C7E0C7F0C800C81D3
:109150000C820C830C840C850C860C870C880C8983
:109160000C8A0C8B0C8C0C8D0C8E0C8F0C900C9133
:109170000C920C930C940C950C960C970C980C99E3
:109180000C9A0C9B0C9C0C9D0C9E0C9F0CA00CA193
:109190000CA20CA30CA40CA50CA60CA70CA80CA943
:1091A0000CAA0CAB0CAC0CAD0CAE0CAF0CB00CB1F3
:1091B0000CB20CB30CB40CB50CB60CB70CB80CB9A3
:1091C0000CBA0CBB0CBC0CBD0CBE0CBF0CC00CC153
:1091D0000CC20CC30CC40CC50CC60CC70CC80CC903
:1091E0000CCA0CCB0CCC0CCD0CCE0CCF0CD00CD1B3
:1091F0000CD20CD30CD40CD50CD60CD70CD80CD963
:109200000CDA0CDB0CDC0CDD0CDE0CDF0CE00CE112
:109210000CE20CE30CE40CE50CE60CE700FE00FEAF
:1092200000FE00FE00FE00FE00FE00FE00FE00FE4E
:1092300000FE00FE00FE00FE00FE00FE00FE00FE3E
:1092400000FE00FE0CE80CE90CEA0CEB0CEC0CED5B
:1092500000FE00FE00FE00FE00FE00FE00FE00FE1E
:1092600000FE00FE00FE00FE00FE00FE00FE00FE0E
:1092700000FE00FE00FE00FE00FE00FE00FE00FEFE
:1092800000FE00FE00FE00FE00FE00FE00FE00FEEE
:1092900000FE00FE00FE00FE00FE00FE00FE00FEDE
:1092A00000FE00FE00FE00FE00FE00FE00FE00FECE
:1092B00000FE00FE00FE00FE00FE00FE00FE00FEBE
:1092C0000CEE0CEF0CF00CF10CF20CF300FE00FEB7
:1092D00000FE00FE00FE00FE00FE00FE00FE00FE9E
:1092E00000FE00FE00FE00FE00FE00FE00FE00FE8E
:1092F00000FE00FE00FE00FE00FE00FE00FE00FE7E
:1093000000FE00FE00FE00FE00FE00FE00FE00FE6D
:1093100000FE00FE00FE00FE00FE00FE00FE00FE5D
:1093200000FE00FE00FE00FE00FE00FE00FE00FE4D
:1093300000FE00FE00FE00FE00FE00FE0CF40CF538
:109340000CF60CF70CF80CF900FE00FE00FE00FE17
:1093500000FE00FE00FE00FE00FE00FE00FE00FE1D
:1093600000FE00FE00FE00FE00FE00FE00FE00FE0D
:1093700000FE00FE00FE00FE00FE00FE00FE00FEFD
:1093800000FE00FE00FE00FE00FE00FE00FE00FEED
:1093900000FE00FE00FE00FE00FE00FE00FE00FEDD
:1093A00000FE00FE00FE00FE00FE00FE00FE00FECD
:1093B00000FE00FE00FE00FE0CFA0CFB0CFC0CFD97
:1093C0000CFE0CFF00FE00FE00FE00FE00FE00FE94
:1093D00000FE00FE00FE00FE00FE00FE00FE00FE9D
:1093E00000FE00FE00FE00FE00FE00FE00FE00FE8D
:1093F00000FE00FE00FE00FE00FE00FE00FE00FE7D
:1094000000FE00FE00FE00FE00FE00FE00FE00FE6C
:1094100000FE00FE00FE00FE00FE00FE00FE00FE5C
:1094200000FE00FE00FE00FE00FE00FE00FE00FE4C
:1094300000FE00FE0AF60AF70AF80AF90AFA0AFB21
:1094400000FE00FE00FE00FE0A7C0A7D0A7E0A7F06
:109450000A8000810A820A830A840A8500FE00FECF
:1094600000FE00FE00FE00FE00FE00FE00FE00FE0C
:1094700000FE00FE00FE00FE00FE00FE00FE00FEFC
:1094800000FE00FE00FE00FE00FE00FE00FE00FEEC
:109490000A860A870A880A890A8A0A8B0A8C0A8D30
:1094A0000A8E0A8F00FE00FE00FE00FE00FE00FE97
:1094B00000FE00FE00FE00FE00FE00FE00FE00FEBC
:1094C00000FE00FE00FE00FE00FE00FE0A900A9173
:1094D0000A920A930A940A950A960A970A980A9990
:1094E0000A9A0A9B0A9C0A9D0A9E0A9F0AA00AA140
:1094F00000FE00FE00EE00FE00FE00FE00FE00FE8C
:1095000000FE00FE00FE00FE00FE00FE00FE00FE6B
:1095100000FE00FE00FE00FE00FE00FE0AA20AA3FE
:109520000AA40AA500FE00FE00FE00FE00FE00FEEA
:1095300000FE00FE00FE00FE00FE00FE00FE00FE3B
:1095400000FE00FE00FE00FE00FE00FE00FE00FE2B
:1095500000FE00FE0AA60AA70AA80AA90AAA0AABE0
:109560000AAC0AAD00FE00FE00FE00FE00FE00FE9A
:1095700000FE00FE00FE00FE00FE00FE00FE00FEFB
:1095800000FE00FE00FE00FE00FE00FE00FE00FEEB
:1095900000FE00FE00FE00FE00FE00FE00FE00FEDB
:1095A00000FE00FE00FE00FE0D000D010D020D0389
:1095B0000D040D050D060D070D080D090D0A0D0B07
:1095C00000FE00FE0D0C0D0D0D0E0D0F0D100D11FA
:1095D0000D120D130D140D150D160D170D180D1977
:1095E0000D1A0D1B0D1C0D1D0D1E0D1F0D200D2127
:1095F0000D220D230D240D250D260D270D280D29D7
:109600000D2A0D2B0D2C0D2D0D2E0D2F0D300D3186
:109610000D320D330D340D350D360D370D380D3936
:109620000D3A0D3B0D3C0D3D0D3E0D3F0D400D41E6
:109630000D420D4300FE00FE00FE00FE00FE00FE97
:1096400000FE00FE0D440D450D460D470D480D4929
:109650000D4A0D4B0D4C0D4D0D4E0D4F0D500D5136
:109660000D520D530D540D550D560D570D580D59E6
:109670000D5A0D5B0D5C0D5D0D5E0D5F0D600D6196
:109680000D620D630D640D650D660D670D680D6946
:109690000D6A0D6B0D6C0D6D0D6E0D6F0D700D71F6
:1096A0000D720D730D740D750D760D770D780D79A6
:1096B0000D7A0D7B0D7C0D7D0D7E0D7F0D800D8156
:1096C0000D820D830D840D850D860D870D880D8906
:1096D0000D8A0D8B0D8C0D8D0D8E0D8F0D900D91B6
:1096E0000D920D9300FE00FE00FE00FE00FE00FE47
:1096F00000FE00FE00FE00FE00FE00FE00FE00FE7A
:1097000000FE00FE00FE00FE00FE00FE0D940D9522
:109710000D960D9700FE00FE00FE00FE00FE00FE0E
:1097200000FE00FE00FE00FE0DA00DA10DA20DA387
:109730000DA40DA50DA60DA700FE00FE0DA80DA9F8
:109740000DAA0DAB0DAC0DAD00FE00FE00FE00FE3F
:109750000DAE0DAF0DB00DB10DB20DB300FE00FE9C
:109760000DB40DB50DB60DB70DB80DB900FE00FE68
:1097700000FE00FE00FE00FE00FE00FE00FE00FEF9
:1097800000FE00FE00FE00FE00FE00FE00FE00FEE9
:1097900000FE00FE00FE00FE00FE00FE00FE00FED9
:1097A00000FE00FE00FE00FE0DC00DC10DC20DC387
:1097B0000DC40DC50DC60DC700FE00FE0DC80DC9B8
:1097C0000DCA0DCB0DCC0DCD00FE00FE00FE00FE3F
:1097D0000DCE0DCF0DD00DD10DD20DD300FE00FE5C
:1097E0000DD40DD50DD60DD70DD80DD900FE00FE28
:1097F00000FE00FE00FE00FE00FE00FE00FE00FE79
:1098000000FE00FE00FE00FE00FE00FE00FE00FE68
:1098100000FE00FE00FE00FE00FE00FE00FE00FE58
:1098200000FE00FE00FE00FE0DE00DE10DE20DE386
:109830000DE40DE50DE60DE700FE00FE0DE80DE977
:109840000DEA0DEB0DEC0DED00FE00FE00FE00FE3E
:109850000DEE0DEF0DF00DF10DF20DF300FE00FE1B
:109860000DF40DF50DF60DF70DF80DF900FE00FEE7
:1098700000FE00FE00FE00FE00FE00FE00FE00FEF8
:1098800000FE00FE00FE00FE00FE00FE00FE00FEE8
:1098900000FE00FE00FE00FE00FE00FE00FE00FED8
:1098A00000FE00FE00FE00FE0AD00AD10AD20AD352
:1098B0000AD40AD50AD60AD700FE00FE0AD80AD969
:1098C0000ADA0ADB0ADC0ADD00FE00FE00FE00FE0A
:1098D0000ADE0ADF0AE00AE10AE20AE300FE00FE0D
:1098E0000AE40AE50AE60AE70AE80AE900FE00FED9
:1098F00000FE00FE00FE00FE00FE00FE00FE00FE78
:1099000000FE00FE00FE00FE00FE00FE00FE00FE67
:1099100000FE00FE00FE00FE00FE00FE00FE00FE57
:1099200000FE00FE00FE00FE0E000E010E020E0301
:109930000E040E050E060E0700FE00FE0E080E09B0
:109940000E0A0E0B0E0C0E0D00FE00FE00FE00FEB9
:109950000E0E0E0F0E100E110E120E1300FE00FE54
:109960000E140E150E160E170E180E1900FE00FE20
:1099700000FE00FE00FE00FE00FE00FE00FE00FEF7
:1099800000FE00FE00FE00FE00FE00FE00FE00FEE7
:1099900000FE00FE00FE00FE00FE00FE00FE00FED7
:1099A00000FE00FE00FE00FE0E200E210E220E2301
:1099B0000E240E250E260E2700FE00FE0E280E2970
:1099C0000E2A0E2B0E2C0E2D00FE00FE00FE00FEB9
:1099D0000E2E0E2F0E300E310E320E3300FE00FE14
:1099E0000E340E350E360E370E380E3900FE00FEE0
:1099F00000FE00FE00FE00FE00FE00FE00FE00FE77
:109A000000FE00FE00FE00FE00FE00FE00FE00FE66
:109A100000FE00FE00FE00FE00FE00FE00FE00FE56
:109A200000FE00FE00FE00FE0E400E410E420E4300
:109A30000E440E450E460E4700FE00FE0E480E492F
:109A40000E4A0E4B0E4C0E4D00FE00FE00FE00FEB8
:109A50000E4E0E4F0E500E510E520E5300FE00FED3
:109A60000E540E550E560E570E580E5900FE00FE9F
:109A700000FE00FE00FE00FE00FE00FE00FE00FEF6
:109A800000FE00FE00FE00FE00FE00FE00FE00FEE6
:109A900000FE00FE00FE00FE00FE00FE00FE00FED6
:109AA00000FE00FE00FE00FE0E600E610E620E6300
:109AB0000E640E650E660E6700FE00FE0E680E69EF
:109AC0000E6A0E6B0E6C0E6D00FE00FE00FE00FEB8
:109AD0000E6E0E6F0E700E710E720E7300FE00FE93
:109AE0000E740E750E760E770E780E7900FE00FE5F
:109AF00000FE00FE00FE00FE00FE00FE00FE00FE76
:109B000000FE00FE00FE00FE00FE00FE00FE00FE65
:109B100000FE00FE00FE00FE00FE00FE00FE00FE55
:109B200000FE00FE00FE00FE0E800E810E820E83FF
:109B30000E840E850E860E8700FE00FE0E880E89AE
:109B40000E8A0E8B0E8C0E8D00FE00FE00FE00FEB7
:109B50000E8E0E8F0E900E910E920E9300FE00FE52
:109B60000E940E950E960E970E980E9900FE00FE1E
:109B700000FE00FE00FE00FE00FE00FE00FE00FEF5
:109B800000FE00FE00FE00FE00FE00FE00FE00FEE5
:109B900000FE00FE00FE00FE00FE00FE00FE00FED5
:109BA00000FE00FE00FE00FE0EA00EA10EA20EA3FF
:109BB0000EA40EA50EA60EA700FE00FE0EA80EA96E
:109BC0000EAA0EAB0EAC0EAD00FE00FE00FE00FEB7
:109BD0000EAE0EAF0EB00EB10EB20EB300FE00FE12
:109BE0000EB40EB50EB60EB70EB80EB900FE00FEDE
:109BF00000FE00FE00FE00FE00FE00FE00FE00FE75
:109C000000FE00FE00FE00FE00FE00FE00FE00FE64
:109C100000FE00FE00FE00FE00FE00FE00FE00FE54
:109C200000FE00FE00FE00FE0EC00EC10EC20EC3FE
:109C30000EC40EC50EC60EC700FE00FE0EC80EC92D
:109C40000ECA0ECB0ECC0ECD00FE00FE00FE00FEB6
:109C50000ECE0ECF0ED00ED10ED20ED300FE00FED1
:109C60000ED40ED50ED60ED70ED80ED900FE00FE9D
:109C700000FE00FE00FE00FE00FE00FE00FE00FEF4
:109C800000FE00FE00FE00FE00FE00FE00FE00FEE4
:109C900000FE00FE00FE00FE00FE00FE00FE00FED4
:109CA00000FE00FE00FE00FE0EE00EE10EE20EE3FE
:109CB0000EE40EE50EE60EE700FE00FE0EE80EE9ED
:109CC0000EEA0EEB0EEC0EED00FE00FE00FE00FEB6
:109CD0000EEE0EEF0EF00EF10EF20EF300FE00FE91
:109CE0000EF40EF50EF60EF70EF80EF900FE00FE5D
:109CF00000FE00FE00FE00FE00FE00FE00FE00FE74
:109D000000FE00FE00FE00FE00FE00FE00FE00FE63
:109D100000FE00FE00FE00FE00FE00FE00FE00FE53
:109D200000FE00FE00FE00FE00FE00FE00FE00FE43
:109D300000FE00FE00FE00FE00FE00FE00FE00FE33
:109D400000FE00FE00FE00FE00FE00FE00FE00FE23
:109D500000FE00FE00FE00FE00FE00FE00FE00FE13
:109D600000FE00FE00FE00FE00FE00FE00FE00FE03
:109D700000FE00FE00FE00FE00FE00FE00FE00FEF3
:109D800000FE00FE00FE00FE00FE00FE00FE00FEE3
:109D900000FE00FE00FE00FE00FE00FE00FE00FED3
:109DA00000FE00FE00FE00FE00FE00FE00FE00FEC3
:109DB00000FE00FE00FE00FE00FE00FE00FE00FEB3
:109DC00000FE00FE00FE00FE00FE00FE00FE00FEA3
:109DD00000FE00FE00FE00FE00FE00FE00FE00FE93
:109DE00000FE00FE00FE00FE00FE00FE00FE00FE83
:109DF00000FE00FE00FE00FE00FE00FE00FE00FE73
:109E000000FE00FE00FE00FE00FE00FE00FE00FE62
:109E100000FE00FE00FE00FE00FE00FE00FE00FE52
:109E200000FE00FE00FE00FE00FE00FE01BB01BCC5
:109E300001BD01BE00B000B100B200B300B400B576
:109E400000B600B700B800B900BA00BB00BC00BD46
:109E500000BE00BF00C000C100C200C300C400C5F6
:109E600000FF00FF00FF00FF00FF00FF02000002F4
:109E7000090270032000000000FFFF00020004023E
:109E80000B0272032258029600B00400020008027E
:109E90000D02740324F4016400D0070002000C02D8
:109EA0000F02760326F4016400D0070002001002BE
:109EB0001102780328F4016400D0070002001402A4
:109EC00013027A032AF4016400D00700020018028A
:109ED00015027C032CF4016400D0070002001C0270
:109EE00017027E032EF4016400D007000200200256
:109EF0001902800330F4016400D00700020024023C
:109F00001B02820332F4016400D007000200280221
:109F10001D02840334F4016400D0070002002C0207
:109F20001F02860336F4016400D0070002003002ED
:109F30002102880338F4016400D0070002003402D3
:109F400023028A033AF4016400D0070001003802BA
:109F500025028C033C0100000002000001003A02CF
:109F600026028D033D0100000002000001003C02BA
:109F700027028E033E0100000002000001003E02A5
:109F800028028F033F010000000200000100400290
:109F9000290290034001000000020000010042027B
:109FA0002A02910341010000000200000100440266
:109FB0002B02920342010000000200000100460251
:109FC0002C0293034301000000020000010048023C
:109FD0002D029403440100000002000001004A0227
:109FE0002E029503450100000002000001004C0212
:109FF0002F029603460100000002000001004E02FD
:10A0000030029703470100000002000002005002E6
:10A010004D024D034864006400D007000100540461
:10A02000DF04DF034A00000000FF000001005604C7
:10A03000E104E1034B00000000FF000000005802B3
:10A0400031023A034C00000000FF000000005902FA
:10A05000320233034D00000000FF000000005A02EE
:10A06000340235034E00000000FF000000005B02D8
:10A07000360237034F00000000FF000000005C02C2
:10A08000380239035000000000FF000000005D06A8
:10A0900000060003515A0020005A000000005E062E
:10A0A00001060103524F0020005A000000005F0625
:10A0B00002060203534E0020005A00000000600612
:10A0C0000306030354450020005A00000000610607
:10A0D0000406040355200020005A00000000620618
:10A0E0000506050356310020005A000000006306F3
:10A0F0000606060357200020005A000000006406F0
:10A100000706070358200020005A000000006506DB
:10A110000806080359200020005A000000006606C7
:10A12000090609035A200020005A000000006706B3
:10A130000A060A035B200020005A0000000068069F
:10A140000B060B035C200020005A0000000069068B
:10A150000C060C035D200020005A000000006A0677
:10A160000D060D035E200020005A000000006B0663
:10A170000E060E035F200020005A000000006C064F
:10A1800010061003605A0020005A000000006D06FF
:10A1900011061103614F0020005A000000006E06F6
:10A1A00012061203624E0020005A000000006F06E3
:10A1B0001306130363450020005A000000007006D8
:10A1C0001406140364200020005A000000007106E9
:10A1D0001506150365320020005A000000007206C3
:10A1E0001606160366200020005A000000007306C1
:10A1F0001706170367200020005A000000007406AD
:10A200001806180368200020005A00000000750698
:10A210001906190369200020005A00000000760684
:10A220001A061A036A200020005A00000000770670
:10A230001B061B036B200020005A0000000078065C
:10A240001C061C036C200020005A00000000790648
:10A250001D061D036D200020005A000000007A0634
:10A260001E061E036E200020005A000000007B0620
:10A27000200620036F5A0020005A000000007C06D0
:10A2800021062103704F0020005A000000007D06C7
:10A2900022062203714E0020005A000000007E06B4
:10A2A0002306230372450020005A000000007F06A9
:10A2B0002406240373200020005A000000008006BA
:10A2C0002506250374330020005A00000000810693
:10A2D0002606260375200020005A00000000820692
:10A2E0002706270376200020005A0000000083067E
:10A2F0002806280377200020005A0000000084066A
:10A300002906290378200020005A00000000850655
:10A310002A062A0379200020005A00000000860641
:10A320002B062B037A200020005A0000000087062D
:10A330002C062C037B200020005A00000000880619
:10A340002D062D037C200020005A00000000890605
:10A350002E062E037D200020005A000000008A06F1
:10A3600030063003A05A0020005A000000008B067F
:10A3700031063103A14F0020005A000000008C0676
:10A3800032063203A24E0020005A000000008D0663
:10A3900033063303A3450020005A000000008E0658
:10A3A00034063403A4200020005A000000008F0669
:10A3B00035063503A5340020005A00000000900641
:10A3C00036063603A6200020005A00000000910641
:10A3D00037063703A7200020005A0000000092062D
:10A3E00038063803A8200020005A00000000930619
:10A3F00039063903A9200020005A00000000940605
:10A400003A063A03AA200020005A000000009506F0
:10A410003B063B03AB200020005A000000009606DC
:10A420003C063C03AC200020005A000000009706C8
:10A430003D063D03AD200020005A000000009806B4
:10A440003E063E03AE200020005A000000009906A0
:10A4500040064003AF5A0020005A000000009A0650
:10A4600041064103B04F0020005A000000009B0647
:10A4700042064203B14E0020005A000000009C0634
:10A4800043064303B2450020005A000000009D0629
:10A4900044064403B3200020005A000000009E063A
:10A4A00045064503B4350020005A000000009F0611
:10A4B00046064603B5200020005A00000000A00612
:10A4C00047064703B6200020005A00000000A106FE
:10A4D00048064803B7200020005A00000000A206EA
:10A4E00049064903B8200020005A00000000A306D6
:10A4F0004A064A03B9200020005A00000000A406C2
:10A500004B064B03BA200020005A00000000A506AD
:10A510004C064C03BB200020005A00000000A60699
:10A520004D064D03BC200020005A00000000A70685
:10A530004E064E03BD200020005A00000000A80671
:10A5400050065003BE5A0020005A00000000A90621
:10A5500051065103BF4F0020005A00000000AA0618
:10A5600052065203C04E0020005A00000000AB0605
:10A5700053065303C1450020005A00000000AC06FA
:10A5800054065403C2200020005A00000000AD060B
:10A5900055065503C3360020005A00000000AE06E1
:10A5A00056065603C4200020005A00000000AF06E3
:10A5B00057065703C5200020005A00000000B006CF
:10A5C00058065803C6200020005A00000000B106BB
:10A5D00059065903C7200020005A00000000B206A7
:10A5E0005A065A03C8200020005A00000000B30693
:10A5F0005B065B03C9200020005A00000000B4067F
:10A600005C065C03CA200020005A00000000B5066A
:10A610005D065D03CB200020005A00000000B60656
:10A620005E065E03CC200020005A00000000B70642
:10A6300060066003CD5A0020005A00000000B806F2
:10A6400061066103CE4F0020005A00000000B906E9
:10A6500062066203CF4E0020005A00000000BA06D6
:10A6600063066303D0450020005A00000000BB06CB
:10A6700064066403D1200020005A00000000BC06DC
:10A6800065066503D2370020005A00000000BD06B1
:10A6900066066603D3200020005A00000000BE06B4
:10A6A00067066703D4200020005A00000000BF06A0
:10A6B00068066803D5200020005A00000000C0068C
:10A6C00069066903D6200020005A00000000C10678
:10A6D0006A066A03D7200020005A00000000C20664
:10A6E0006B066B03D8200020005A00000000C30650
:10A6F0006C066C03D9200020005A00000000C4063C
:10A700006D066D03DA200020005A00000000C50627
:10A710006E066E03DB200020005A00000000C60613
:10A7200070067003DC5A0020005A00000000C706C3
:10A7300071067103DD4F0020005A00000000C806BA
:10A7400072067203DE4E0020005A00000000C906A7
:10A7500073067303DF450020005A00000000CA069C
:10A7600074067403E0200020005A00000000CB06AD
:10A7700075067503E1380020005A00000000CC0681
:10A7800076067603E2200020005A00000000CD0685
:10A7900077067703E3200020005A00000000CE0671
:10A7A00078067803E4200020005A00000000CF065D
:10A7B00079067903E5200020005A00000000D00649
:10A7C0007A067A03E6200020005A00000000D10635
:10A7D0007B067B03E7200020005A00000000D20621
:10A7E0007C067C03E8200020005A00000000D3060D
:10A7F0007D067D03E9200020005A00000000D406F9
:10A800007E067E03EA200020005A00000000D506E4
:10A8100080068003EB5A0020005A00000000D60694
:10A8200081068103EC4F0020005A00000000D7068B
:10A8300082068203ED4E0020005A00000000D80678
:10A8400083068303EE450020005A00000000D9066D
:10A8500084068403EF200020005A00000000DA067E
:10A8600085068503F0390020005A00000000DB0651
:10A8700086068603F1200020005A00000000DC0656
:10A8800087068703F2200020005A00000000DD0642
:10A8900088068803F3200020005A00000000DE062E
:10A8A00089068903F4200020005A00000000DF061A
:10A8B0008A068A03F5200020005A00000000E00606
:10A8C0008B068B03F6200020005A00000000E106F2
:10A8D0008C068C03F7200020005A00000000E206DE
:10A8E0008D068D03F8200020005A00000000E306CA
:10A8F0008E068E03F9200020005A00000000E406B6
:10A9000090069005605A0020005A00000000E506FD
:10A9100091069105614F0020005A00000000E606F4
:10A9200092069205624E0020005A00000000E706E1
:10A930009306930563450020005A00000000E806D6
:10A940009406940564200020005A00000000E906E7
:10A950009506950565310020005A00000000EA06C2
:10A960009606960566300020005A00000000EB06AF
:10A970009706970567200020005A00000000EC06AB
:10A980009806980568200020005A00000000ED0697
:10A990009906990569200020005A00000000EE0683
:10A9A0009A069A056A200020005A00000000EF066F
:10A9B0009B069B056B200020005A00000000F0065B
:10A9C0009C069C056C200020005A00000000F10647
:10A9D0009D069D056D200020005A00000000F20633
:10A9E0009E069E056E200020005A00000000F3061F
:10A9F000A006A0056F5A0020005A00000000F406CF
:10AA0000A106A105704F0020005A00000000F506C5
:10AA1000A206A205714E0020005A00000000F606B2
:10AA2000A306A30572450020005A00000000F706A7
:10AA3000A406A40573200020005A00000000F806B8
:10AA4000A506A50574310020005A00000000F90693
:10AA5000A606A60575310020005A00000000FA067F
:10AA6000A706A70576200020005A00000000FB067C
:10AA7000A806A80577200020005A00000000FC0668
:10AA8000A906A90578200020005A00000000FD0654
:10AA9000AA06AA0579200020005A00000000FE0640
:10AAA000AB06AB057A200020005A00000000FF062C
:10AAB000AC06AC057B200020005A00000001000617
:10AAC000AD06AD057C200020005A00000001010603
:10AAD000AE06AE057D200020005A000000010206EF
:10AAE000B006B0057E5A0020005A0000000103069F
:10AAF000B106B1057F4F0020005A00000001040696
:10AB0000B206B205804E0020005A00000001050682
:10AB1000B306B30581450020005A00000001060677
:10AB2000B406B40582200020005A00000001070688
:10AB3000B506B50583310020005A00000001080663
:10AB4000B606B60584320020005A0000000109064E
:10AB5000B706B70585200020005A000000010A064C
:10AB6000B806B80586200020005A000000010B0638
:10AB7000B906B90587200020005A000000010C0624
:10AB8000BA06BA0588200020005A000000010D0610
:10AB9000BB06BB0589200020005A000000010E06FC
:10ABA000BC06BC058A200020005A000000010F06E8
:10ABB000BD06BD058B200020005A000000011006D4
:10ABC000BE06BE058C200020005A000000011100C6
:10ABD000550055058D000000000100000001120223
:10ABE0006C029C058F0300010009000000011302A4
:10ABF0006D029D05900A000000140000000114027F
:10AC00006E029E0591140000001000000103FE0278
:10AC10000302FE058EC3000000FF00000000C1C05B
:10AC200081C1400101C3C003800241C201C6C00608
:10AC3000800741C70005C1C581C4400401CCC00CD8
:10AC4000800D41CD000FC1CF81CE400E000AC1CA98
:10AC500081CB400B01C9C009800841C801D8C01888
:10AC6000801941D9001BC1DB81DA401A001EC1DE08
:10AC700081DF401F01DDC01D801C41DC0014C1D4F8
:10AC800081D5401501D7C017801641D601D2C01218
:10AC9000801341D30011C1D181D0401001F0C030E8
:10ACA000803141F10033C1F381F240320036C1F608
:10ACB00081F7403701F5C035803441F4003CC1FCD8
:10ACC00081FD403D01FFC03F803E41FE01FAC03A98
:10ACD000803B41FB0039C1F981F840380028C1E8C8
:10ACE00081E9402901EBC02B802A41EA01EEC02E08
:10ACF000802F41EF002DC1ED81EC402C01E4C024F8
:10AD0000802541E50027C1E781E640260022C1E217
:10AD100081E3402301E1C021802041E001A0C06027
:10AD2000806141A10063C1A381A240620066C1A607
:10AD300081A7406701A5C065806441A4006CC1ACD7
:10AD400081AD406D01AFC06F806E41AE01AAC06A97
:10AD5000806B41AB0069C1A981A840680078C1B887
:10AD600081B9407901BBC07B807A41BA01BEC07E07
:10AD7000807F41BF007DC1BD81BC407C01B4C074F7
:10AD8000807541B50077C1B781B640760072C1B217
:10AD900081B3407301B1C071807041B00050C19067
:10ADA000819140510193C053805241920196C05607
:10ADB000805741970055C19581944054019CC05CD7
:10ADC000805D419D005FC19F819E405E005AC19A97
:10ADD000819B405B0199C059805841980188C048C7
:10ADE00080494189004BC18B818A404A004EC18E07
:10ADF000818F404F018DC04D804C418C0044C184F7
:10AE0000818540450187C047804641860182C04216
:10AE1000804341830041C18181804040FFFFFFFFAB
:02AE2000FFFF32
:00000001FF
